:020000040000FA
:10000000D3EF01F01200FFFF04EF04F01200FFFF36
:100010001500FFFFFFFFFFFF0CEF04F01200FFFFD2
:10002000F26A1AEF01F0120000001200C3EC01F0B6
:10003000C3EC01F0C3EC01F0C3EC01F0C3EF01F03D
:10004000C80EF46EC3EC01F087B0000CF406F45057
:100050000008F8E3010CA7EC01F0E8DF9194000E32
:10006000F66E080EF76E0900F5CF07F00800F5CF21
:1000700008F00750081004E062EC00F0000903E00B
:10008000DFDF000903E01AEF01F005D091688B80F3
:100090008B8401EF04F01200F66A080EF76EF86A1E
:1000A0000DD8800EF626000EF722F822800EF65CA0
:1000B000FD0EF758010EF858F3E31200940E7F6E10
:1000C000B1EF00F0D9CFE6FFE1CFD9FF020EE12674
:1000D000D9CFE9FFDACFEAFFEE6AED6AF66A080ED9
:1000E000F76EF86A0900F550F46E0900F550F36EEA
:1000F000D9CFE9FFDACFEAFFF350EE26F450ED2234
:10010000F350F41002E1010E20D00900F550F46E16
:100110000900F550F36ED9CFE9FFDACFEAFFF350CB
:10012000EE26F450ED22800EF65CFD0EF758010E1F
:10013000F858EBE3D9CFE9FFDACFEAFFEE50ED1044
:1001400002E0000E01D0010E00D0076E020EE15C4D
:1001500002E2E16AE552E16E0750E552E7CFD9FFCE
:100160001200550E7E6EAA0E7E6E7F8200007F9476
:100170001200010EF46E0A00800EF36EEE50F56E62
:100180000F00F306F3500008F9E3840E7F6EE9DFF9
:10019000F406F4500008F0E31200610EE96E000E60
:1001A000EA6EB9EF00F0FF0012009CEC01F09EAA8D
:1001B000FCD783EC01F00009F8E0490E005C0DE18A
:1001C0006B0E7FD8610E7DD8740E7BD8350E79D832
:1001D000300E77D8300E75D8E8D70050AD6E440E8B
:1001E000005CE3E112000001E151076E07507F0B54
:1001F00001E0000CE1C0F6FFE2C0F7FFE3C0F8FF4A
:10020000010CF46A610EE96E000EEA6E9EAAFED73A
:1002100083EC01F0000901E1000C0050EF6EEE509C
:10022000F426E50EE95C000EEA58F0E3F45001E034
:10023000000C010C0001606BA7EC01F091866BECE7
:1002400001F0B3DF9184016A026ADBDF000903E099
:10025000CADF000902E14E0E1ED0020EF85C0AE170
:10026000F66A080EF76EF86A5EEC00F096DF420E52
:10027000AD6E21D0000EF65C080EF758000EF8584F
:1002800002E2410E08D0800EF65CFD0EF758010E1A
:10029000F85803E34E0EAD6ED8D70001605105E16A
:1002A000010E606F4CEC00F09EDF77DF410EAD6E0B
:1002B00091EC01F0CAD7ACA2FED7BEEC01F0D3EFAF
:1002C00000F0E66E76EC01F0E55212009EAA02D034
:1002D000AE50FCD71200040EAC6E100EAB6E656A09
:1002E000190EAF6EAC8AAB8E66EF01F0D9CFE6FF88
:1002F000E1CFD9FFACA2FED7FE0EDB50AD6EE552CA
:10030000E7CFD9FF12009EAA0BD0ABA204D0AB98C6
:10031000DDDFAB88F8D7AE50006EABB4F4D7010C7C
:10032000000CBEEC01F0012A000E022201A802D04E
:100330009196120091861200BEEC01F0012A000E87
:10034000022202AA02D091941200918412000F019D
:10035000010E256F246B700E236F050E8B6E8E6A57
:100360008F6A200E906E9168900E946E700E976E4C
:10037000200E986E0B0E996E9A6A1200140E036E80
:10038000046AC9EF01F0200E036E4E0E046EC9EF31
:1003900001F00306000E045A0350041003E00000AD
:1003A0000000F7D712001EEE00F02EEE00F0F86A03
:1003B000069C32EC02F0E3EC01F015EC00F02BECC3
:1003C00000F0FBD71200280EF66E000EF76E000E3E
:1003D000F86E0F010900F550056F0900F550066F22
:1003E00003E1056701D03DD00900F550006F090019
:1003F000F550016F0900F550026F09000900F55032
:10040000E96E0900F550EA6E090009000900F5508F
:10041000036F0900F550046F09000900F6CF07FFCC
:10042000F7CF08FFF8CF09FF00CFF6FF01CFF7FFA6
:1004300002CFF8FF0F01035302E1045307E0090064
:10044000F550EE6E0307F8E20407F9D707CFF6FF81
:1004500008CFF7FF09CFF8FF0F010507000E065B75
:10046000BFD71200160EF36E00EE00F00F0E01D88B
:100470001200EA6002D0EE6AFCD7F350E960120085
:10048000EE6AFCD7FFFFFFFFFFFFFFFFFFFFFFFF4D
:10049000FFFFFFFFFFFFFFFFFFFFFFFFFFFFFFFF6C
:1004A000FFFFFFFFFFFFFFFFFFFFFFFFFFFFFFFF5C
:1004B000FFFFFFFFFFFFFFFFFFFFFFFFFFFFFFFF4C
:1004C000FFFFFFFFFFFFFFFFFFFFFFFFFFFFFFFF3C
:020800000000F6
:0608020077EF4BF012003D
:04080800DDEF3BF0F5
:0408180013EF45F0A5
:1008200002008D970000BD050000160000008C97A7
:0A0830000000C406000001000000F3
:06083A000501200E9F6F76
:100840000D0EA06F020E0301912588EC0AF0030142
:10085000922145EC0AF001E11200050E03019EEC25
:100860000AF03AEC0AF00AE1040E9EEC0AF0EA22E1
:10087000EFCF10F620CD0FF6B3EF20F0060E9EEC72
:100880000AF03AEC0AF012E1050E9EEC0AF05CEC7C
:100890000AF007E0010A01E012000401786B52EF50
:1008A0000AF00401010E786F52EC0AF01200050103
:1008B000440E9F6F0D0EA06F030E0301932588EC6D
:1008C0000AF00301942145EC0AF001E11200050E43
:1008D0000301C4EC0AF004E144CD13F6FFEF20F06D
:1008E000060EC4EC0AF018E1050EEA6A9325E96EDB
:1008F00094515CEC0AF009E0010A01E012000401E5
:10090000906B44CD8FF4C7EF0EF00401010E906F91
:1009100044CD8FF4C7EC0EF01200030E0301CAECB5
:100920000AF00EE10601410E42EC0AF0480E42ECDC
:100930000AF0340E3FEC0BF007C48CF679EF0AF0A6
:1009400090EC0AF0EF504B0806E195C397F396C37D
:1009500098F3B6EF04F0040ECAEC0AF006E190EC4E
:100960000AF0EFCF4FF446EC20F01200040E030122
:10097000D0EC0AF002E1C3EF49F0050ED0EC0AF02A
:1009800014E1040EEA6A9725E96E98515CEC0AF0CE
:1009900007E0010A01E012000601C36BE0EF49F035
:1009A0000601010EC36FE0EC49F01200040E0301D2
:1009B000EA6A9925E96E9A513AEC0AF002E1F0EF01
:1009C00039F0040E99254BEC0AF003019A213EEC14
:1009D0000AF0F3CF45F4F4CF46F49DEF1FF0040E78
:1009E0000301D6EC0AF002E149EF43F0050ED6EC24
:1009F0000AF018E18CEC0AF015E1040E0301EA6A32
:100A00009B25E96E9C515CEC0AF005E0010A01E0CF
:100A10001200FCEF42F0060173870601BC6BBD6B50
:100A20001FEC43F01200020E0301A9EC0AF05CEC8B
:100A30000AF01EE0030A1CE0010A1AE0030A05E0BE
:100A40000B0A01E0120040EF48F0030EA9EC0AF097
:100A50003AEC0AF01CE104015651030B0401826FC9
:100A60005DC481F4BEEC0DF00501FD6FFC81120048
:100A7000030EA9EC0AF03AEC0AF009E1020EA9EC27
:100A80000AF0EA22EF50030B0501FD6FFC81120012
:100A90000501200E9F6F0D0EA06F020E03019F2512
:100AA00088EC0AF00301A02145EC0AF001E11200F4
:100AB000040E0301DCEC0AF0300A0DE0010A0BE041
:100AC000030A09E0010A07E0080A01E0120020CD4C
:100AD00015F6DCEF21F0050EEA6A9F25E96EA051BC
:100AE0003AEC0AF00AE1040EDCEC0AF0030B040114
:100AF000926F20CD91F430EC0FF01200040E030140
:100B0000E3EC0AF002E162EF47F0050EE3EC0AF0D5
:100B100013E197EC0AF010E1040E0301EA6AA12543
:100B2000E96EA2515CEC0AF005E0010A01E0120056
:100B30002FEF47F034EC47F0120061EF4AF0020E5D
:100B4000BDEC0AF004E103C467F695EF3AF0050145
:100B5000020E9F6F0D0EA06F020E0301A32588ECFD
:100B60000AF00301A42145EC0AF001E112000B0E8A
:100B70000D01025D01E31200040EBDEC0AF001E07C
:100B8000120002CD80F486EC0DF060EF0AF0020E48
:100B90000301AEEC0AF03AEC0AF004E104C4B3F647
:100BA000AAEF4AF0030EAEEC0AF03AEC0AF023E1A9
:100BB000020EAEEC0AF0EA22EF50330A10E0010A0E
:100BC0000BE0030A06E0010A01E012000401CF0E67
:100BD00008D00401670E05D00401330E02D00401D1
:100BE000190E056F020E0301AEEC0AF0EA22EFCFF8
:100BF00004F4ABEC46F01200030E0301E9EC0AF03A
:100C000002E16FEF49F0040EE9EC0AF011E1030E86
:100C1000EA6AA725E96EA851EA22EF504E0A06E0DB
:100C20000C0A01E012000401569F12000401568FC5
:100C30001200010E0301EFEC0AF002E10EEF4BF09F
:100C4000030EEFEC0AF014E18CEC0AF011E105015F
:100C5000570EA36F040EA46F010E0301A925050111
:100C6000A16F000E0301AA210501A26F5AEC2AF020
:100C700012008CEC0AF002E00501FC851200020E65
:100C80000301AB254BEC0AF00301AC21F7DBF3CFFA
:100C900000F6F4CF01F641EF34F08CEC0AF009E1F4
:100CA00097EC0AF006E1F8EC3FF091EC1EF0EEEC68
:100CB00042F01200050E0301EA6AAD25E96EAE515D
:100CC000D9DB01E012008CEC0AF001E01200050112
:100CD0000A0E9F6F0D0EA06F020E0301AD2588EC6A
:100CE0000AF00301AE21D1DB01E11200040E030181
:100CF000EA6AAD25E96EAE51EA22EF50030B03011B
:100D0000736F0ACD72F348EF12F0010E0301AF25A5
:100D1000C2DB0301B021B2DBF3CF04FDF4CF05FD4C
:100D20000D01F350F41006E13FC679F640C67AF69D
:100D3000C4EF48F004CDA1F605CDA2F690EF42F045
:100D4000020E0301C3DB01E01200030EBFDB01E072
:100D50001200040EBBDB01E0120005010B0E966FC2
:100D6000020E0301B1250501946F000E0301B221AB
:100D70000501956FC8EC29F0000901E112000D0E84
:100D800003012BEC0BF076DB01E012000A0E2BECDA
:100D90000BF0EA22EF6A050EB1257DDB0301B221DB
:100DA0006DDB8ED305017651000806E2AFEC1EF034
:100DB000F8EC27F0EEEC42F01200040E0301EA6AB0
:100DC000B325E96EB45156DB0FE1030EEA6AB32591
:100DD000E96EB45171DB06E0010A01E01200060180
:100DE00073911200060173811200030E0301F5ECEA
:100DF0000AF002E18FEF3BF0030EEA6AB525E96ED7
:100E0000B651EA22EF50430807E1040EEEDB04E19D
:100E10000601A06BA6EC3BF01200030E0301B72500
:100E20003ADB0301B8212ADBF3CF04FDF4CF05FD43
:100E30000501765100080DE20501020EFA6F050169
:100E4000040EF86F0D0EF96F0501F66BF76B44ECAD
:100E50003FF012000601470E15DB4F0E3FEC0BF082
:100E600024C60CFF25C60DFFB5EC33F049EF33F077
:100E700006014B0E07DB410E05DB540E03DB350E7E
:100E800001DB300EFFDA300E8C6F33D3010E03011D
:100E9000B2DB02E1F3EF45F0030EADDB13E13CDB27
:100EA00011E10501580EA36F040EA46F010E03019A
:100EB000B9250501A16F000E0301BA210501A26F3A
:100EC0005AEC2AF01200020E03014DDBD3DA02E1E4
:100ED0005AEF39F0030E47DBCDDA17E1020E43DBA0
:100EE000EA22EF50550A0AE0140A05E0030A03E07B
:100EF0000F0A01E01200020E73EF0AF005017651AD
:100F0000000803E2020E0301EEDA1200020E0301F2
:100F1000BD25C1DA0301BE21B1DAD2D2030E03012D
:100F200070DB02E14CEF39F0040E6BDB13E1030ED2
:100F3000EA6ABF25E96EC051BFDA07E0010A01E0A5
:100F400012000401486BBFEF1FF00401010E486F4F
:100F5000BFEC1FF01200030E030159DB02E153EF57
:100F600039F0040E54DB13E1030EEA6AC125E96E81
:100F7000C251A2DA07E0010A01E012000401496B44
:100F8000C6EF1FF00401010E496FC6EC1FF01200FE
:100F9000020E030142DB02E105EF47F0030E3DDBE9
:100FA0000FE1020EEA6AC325E96EC45185DA06E054
:100FB000010A01E012000601C28D12000601C28F73
:100FC0001200030E03012FDB02E143EF39F0040EA0
:100FD0002ADB13E1030EEA6AC525E96EC6516CDA15
:100FE00007E0010A01E012000401476BB8EF1FF0AF
:100FF0000401010E476FB8EC1FF01200030E03014D
:10100000EA6AC725E96EC851EA22EF50300A07E0C4
:10101000010A01E0120090EC10F08DEC20F0EEEFF0
:1010200042F00601520E2EDA560E2CDA300E2ADA73
:10103000310E28DA2E0E26DA360E24DA330E8C6FB5
:1010400058D2040E0301F5DA02E136EF49F0050E3D
:10105000F0DA11E1040EEA6AC925E96ECA51EA2202
:10106000EF50540A06E0150A01E012000401568D03
:1010700012000401569D1200020E0301E0DA02E1A3
:101080007FEF39F0030EDBDA13E1020EEA6ACB25BB
:10109000E96ECC5111DA07E0010A01E01200040107
:1010A0004B6BE3EF1FF00401010E4B6FE3EC1FF0FD
:1010B0001200020E0301CD25EED90301CE21DED9A7
:1010C000F3CF20FDF4CF21FD0D01F350F41004E126
:1010D0003FC620FD40C621FDC2EC1CF0000906E021
:1010E000E6EC3DF0F3CF20FDF4CF21FD15DA06E16B
:1010F00020CDAAF621CDABF620EC4AF012000D016E
:10110000236B246B256B266B0501220E9F6F0D0E42
:10111000A06F020E0301CF25FBD90301D021B5D961
:1011200001E11200050E03019BDAA4D909E1040EC6
:1011300097DAEA22EFCF19F622CD18F6F9EF21F06F
:10114000050ECF250D01276F000E0301D0210D01E3
:10115000286F8BDAD2D905E00D01272B000E28234A
:10116000F8D79DD918E00D010A0E2403F3CF24FD12
:101170002303F3CF23FDF4502427B2D9D00F146EEC
:10118000156A14BE15681450232715502423272BE5
:10119000000E2823E6D7A4D92E081FE10D01272B26
:1011A000000E28237CD919E09BD9D00F0A0DF3CF6C
:1011B00025FD0D01266B25BF2669272B000E282350
:1011C0006ED90BE08DD9D00F146E156A14BE156858
:1011D00014500D012527155026230D01010E235D06
:1011E000000E245901E21200630ED8802355000E30
:1011F000245501E2120025CD05FF15EC33F00D0159
:10120000256F23CD26FDE8CF95F423CD96F4040E6B
:10121000030126DAEA22EFCF94F422CD93F4ABEF68
:101220000FF0030E0301D12536D90301D22126D9AF
:10123000F3CF44F5F4CF45F575EF2CF0020E030122
:1012400097D918D90BE10601540E1CD9450E17DAAF
:1012500000C508FF57EC33F049EF33F0040E88D98E
:1012600009D921E10501020E996F0301D32505017A
:10127000976F000E0301D4210501986FD8EC29F077
:10128000000911E0030E030173D9EA22EFCF93F5B1
:10129000020E6ED9EA22EFCF92F5B9EC29F00501E2
:1012A000096FB7EC22F01200030E0301D525F3D825
:1012B0000301D621E3D8F3CF54F5F4CF55F517EF5A
:1012C0002DF0030E0301D725E6D80301D821D6D887
:1012D000F3CF56F5F4CF57F52FEF2DF047EF2DF064
:1012E000030E0301DB25D7D80301DC21C7D8F3CFD8
:1012F00046F5F4CF47F581EF2CF0030E0301DD2511
:10130000CAD80301DE21BAD8F3CF48F5F4CF49F5A6
:1013100090EF2CF00601540EB5D8500EB0D9A1ECC8
:1013200035F00F010A6F6DEC33F049EF33F0030E27
:101330000301DF25B0D80301E021A0D8F3CF4EF59B
:10134000F4CF4FF5D5EF2CF0030E03017ED903E166
:1013500003C444FD11D0050E78D912E10501440EF5
:101360009F6F0D0EA06F030E0301E125D1D803017D
:10137000E2218BD801E1120044CD14F65EEC21F09D
:101380001200030E0301E32586D80301E42176D879
:10139000F3CF4CF5F4CF4DF5B5EF2CF0030E030170
:1013A000E52579D80301E62169D8F3CF51F5F4CFCB
:1013B00052F5EFEF2CF0030E0301E7256CD8030183
:1013C000E8215CD8F3CF53F5FAEF2CF0030E0301BC
:1013D00051D950D807E1020E4DD9EA22EFCFC1F61C
:1013E00088EF39F0030EE92556D80301EA2146D8E3
:1013F000F3CF4DF4F4CF4EF4020E03013BD9EA22B1
:10140000EFCF4CF4EAEF1FF0020E0301EB250D01C4
:10141000006F000E0301EC210D01016F0601696BE5
:1014200006016A6B58D869D802E06DD8FBD753D84B
:101430008AD80BE00A0E06016903F3CF69F64BD890
:10144000EF50D00F69275FD8F2D745D856D802E0C1
:101450005AD8FBD740D877D80BE00A0E06016A03AA
:10146000F3CF6AF638D8EF50D00F6A274CD8F2D7AE
:1014700098EF31F0EA22EF503B0812000501A66F09
:1014800075EF2AF0FCD80601120005019E6F3FECB3
:101490002AF0000912000501A56F000E1200E5D820
:1014A000A3EF0AF0040E030149D8EA22EFCF77F444
:1014B00020CD76F4AFEF0BF0EA22EF50310A1200A4
:1014C000F3CFA1F6F4CFA2F690EF42F0C4D8EA220F
:1014D000EF503008120000CDE9FF01CDEAFF120005
:1014E000C4D8EF5012003FD8EA22EFCF4AF4CDEF34
:1014F0001FF0C3EC46F049EF33F0EFCF9CF535EC2D
:101500002AF0000912000D01002B000E0123120029
:1015100005019D6F000E1200A1EC35F000091200CC
:10152000030EEA6A9525E96E9651EA22120004013B
:10153000F66BF76B26EC1DF000091200EA6A9125A4
:10154000E96E92511200EFCF9AF5E8EC29F000090C
:101550001200EA6A9D25E96E9E511200EA6AA525ED
:10156000E96EA6511200EA6ABB25E96EBC51120071
:10157000EA6AD325E96ED45112000301EA6AA32571
:10158000E96EA4513AEF0AF0EA6A9325E96E9451A4
:101590003AEF0AF0EA6A9525E96E96513AEF0AF0B9
:1015A000EA6A9725E96E98513AEF0AF0EA6A9B25B4
:1015B000E96E9C513AEF0AF0EA6A9F25E96EA05164
:1015C000EA22EF501200EA6AA125E96EA2513AEF31
:1015D0000AF0EA6AA725E96EA8513AEF0AF0EA6A2A
:1015E000A925E96EAA513AEF0AF0EA6AB525E96E33
:1015F000B6513AEF0AF0EA6AB925E96EBA513AEF04
:101600000AF0EA6ABF25E96EC0513AEF0AF0EA6AC9
:10161000C125E96EC2513AEF0AF0EA6AC325E96EC4
:10162000C4513AEF0AF0EA6AC525E96EC6513AEFAD
:101630000AF0EA6AC925E96ECA513AEF0AF0EA6A85
:10164000CB25E96ECC513AEF0AF0EA6AE125E96E62
:10165000E2513AEF0AF0EA6AB125E96EB25112009E
:10166000EA6ACF25E96ED051120027CDE9FF28CDD7
:10167000EAFF1200EA6AE925E96EEA5112008C6F6E
:04168000C3EF46F07E
:0C1684008BEC11F00401826F1EEC11F0E1
:101690006DEC11F00D01226F8BEC11F0225D01E178
:1016A000000C8BEC11F0146E1EEC11F00E0EEB50D2
:1016B000145C0CE11EEC11F0030EEB5004019C6F66
:1016C00070C49AF471C49BF4DFEC10F00D01225148
:1016D000146E1EEC11F082EC11F0010C550E040199
:1016E000085D26E054EC11F07DEC11F00601BB6FB3
:1016F00054EC11F02BEC11F01BE154EC11F00D0E39
:1017000013EC11F0EF500501196F1A6B54EC11F046
:101710007DEC11F00501176F186BA30E0501156F15
:10172000166B62EC23F072C470F473C471F4AADF18
:10173000120038EC11F000090CE038EC11F0060151
:10174000BB6F2BEC11F005E038EC11F0146E82EF5A
:1017500011F074C472F475C473F46EEF0BF00B0ED9
:101760000401765D01E31200040103510401765D7A
:1017700047E150C400FD51C401FD52C402FD53C4F1
:1017800003FD54C404FD55C405FD56C406FD57C4ED
:1017900007FD58C408FD59C409FD5AC40AFD5BC4BD
:1017A0000BFD5CC40CFD5DC40DFD5EC40EFD5FC48D
:1017B0000FFD60C410FD61C411FD62C412FD63C45D
:1017C00013FD64C414FD65C415FD66C416FD67C42D
:1017D00017FD68C418FD69C419FD6AC41AFD6BC4FD
:1017E0001BFD6CC41CFD6DC41DFD6EC41EFD6FC4CD
:1017F0001FFD0401000E886F0D0E896F1ADA08D0E4
:1018000076C48CF40401000E8A6F0D0E8B6F40DAE3
:101810000401785111E07751330A0BE0010A06E028
:10182000030A01E012000D010D8116D00D010D8398
:1018300013D00D010D8510D07751330A0BE0010A4A
:1018400006E0030A01E012000D010D9105D00D0123
:101850000D9302D00D010D950E5110E00ECDBBF68B
:101860000DCDBAF666EC4BF0000908E10D010E6BE8
:101870000401000E726F0D0E736F30DF0D01065103
:1018800045EC11F00DE10401000E846F0D0E856F23
:101890009AD90D01030BF36EFC0E0615F310066FBB
:1018A00076C49CF40401000E9A6F0D0E33EC11F017
:1018B0000401765D1AE10DCD5DF40ECD5EF4565156
:1018C00045EC11F012E10401500E846F040E856F97
:1018D0007AD90401030BF36EFC0E5615F310566F04
:1018E000E850030B0501FD6FFC8112000B0E040193
:1018F000795D01E31200040103510401795D41E1C6
:1019000050C400FD51C401FD52C402FD53C403FD87
:1019100054C404FD55C405FD56C406FD57C407FD57
:1019200058C408FD59C409FD5AC40AFD5BC40BFD27
:101930005CC40CFD5DC40DFD5EC40EFD5FC40FFDF7
:1019400060C410FD61C411FD62C412FD63C413FDC7
:1019500064C414FD65C415FD66C416FD67C417FD97
:1019600068C418FD69C419FD6AC41AFD6BC41BFD67
:101970006CC41CFD6DC41DFD6EC41EFD6FC41FFD37
:1019800008D079C48CF40401000E8A6F0D0E8B6FA1
:101990007FD904017B5111E07A51330A0BE0010A2F
:1019A00006E0030A01E012000D010D8B16D00D01B7
:1019B0000D8D13D00D010D8F10D07A51330A0BE02D
:1019C000010A06E0030A01E012000D010D9B05D09B
:1019D0000D010D9D02D00D010D9F0DCD24F579C493
:1019E00023F50501F00E216F260E226FA8EC23F0DF
:1019F00079C49CF40401000E9A6F0D0E33EC11F0C3
:101A00000401795D02E10DCD5DF41200200EE66E59
:101A1000E66ACC0EE66E7CC4E6FF7DC4E6FF20ECF1
:101A20004BF0146E050EE15E1450F8DB200E8EECC8
:101A300011F0EE52030E8EEC11F0020EF4DBA40E48
:101A40008EEC11F0030E7EC4EBFFE8DB040EEB6AB4
:101A5000050EEB6A79EC11F0EF6A79EC11F0EF9E6C
:101A600079EC11F0EF9C79EC11F0FC0EEF14010908
:101A7000EF6E79EC11F0EE52EF6A79EC11F0020E94
:101A8000D2DBEF6A79EC11F0030ECDDBEE68630E6A
:101A9000ED6EC4DB0C0EC7DB410E8EEC11F00D0EAB
:101AA000C2DB070E8EEC11F00E0EBDDBEF6AB6DB6B
:101AB0000F0EB9DB330E86EC11F0110EB4DBCD0E38
:101AC00086EC11F0130EAFDBEE6A030EED6EA6DBB3
:101AD000180EA9DB9A0E86EC11F0170EA4DBEF6A44
:101AE00012000401035104017F5D03E15DC400FDA8
:101AF0000AD07F51200DF3CFECF5F4CFEDF58D0E2C
:101B0000F2DB0D01006F0D010051120004010351C1
:101B10000401805D05E154C400FD55C401FD0DD0F4
:101B20000501020EF56F0501000EF36F0D0EF46F47
:101B300004018051B3DB840EA2DB0D0100510111C1
:101B400008E180C466F65FEC3AF0F3CF00FDF4CF15
:101B500001FD00CD19F501CD1AF5040180510501F3
:101B6000176F186B0501E70E156F030E166F62EC09
:101B700023F000CDF3FF01CDF4FF120004018251E8
:101B8000020A07E0030A0AE181B3020C81B5030CE3
:101B9000010C81B5030C81B1010C020C81B1010C67
:101BA00081B3020C030C040103510401835D02E1C3
:101BB0005E5112008351200DF3CFECF5F4CFEDF51B
:101BC0008E0E73EF11F033DB000907E030DB060106
:101BD000BB6F41DB02E017EF11F029DB0401826FDC
:101BE0006DEF11F04CD868C431F669C432F636ECAA
:101BF00030F0000905E104019A0E686F010E696F6B
:101C00000401000E635D010E645905E3000E635D7F
:101C1000630E645903E3636B030E646F90EF10F07F
:101C200087C4BBF686C47FF45CDF0601BA6F66EF3B
:101C30004BF03FDB0E0EEB50000916E03ADB0E0EC8
:101C4000EB50146E5ADB145C0FE00501060EF56FC5
:101C500030DBE9DAE9CFF3F5EACFF4F52ADB030E5E
:101C6000EB501CDB860E0BDB12000401569D569FC9
:101C7000576B586B2BC659F42CC65AF4120003C488
:101C80008CF40401500E8A6F040E8B6F48EF0EF037
:101C90000B0E04018C5D01E312000501200EF56FAF
:101CA0008AC4F3F58BC4F4F504018C51F7DA800E85
:101CB000E6DA8CC499F48AC497F48BC498F406DAF3
:101CC000000916E10501196B1A6B04018C5105011D
:101CD000176F186B700E0501156F166B62EC23F011
:101CE0008CC47EF48AC47CF48BC47DF406EF0DF0C2
:101CF000E5DA0E0EEB50000918E0E0DA0E0EEB50BC
:101D0000146E00DBDBDA110E8EDAEECF14F0EFCFBB
:101D100015F0800E145C010E155807E2CFDA110E93
:101D200082DA800EEE6E010EED6E1200CCDAEF500C
:101D3000800B01E0010E0601B96F77EC49F00D014F
:101D4000006FC1DAEF50400B01E0010E0601B16FE8
:101D50003BEC49F00D010013B6DA010EEB50060121
:101D6000B76F12EC4BF00D010013ADDA020EEB5021
:101D70000601B56FF8EC45F00D010013005112009B
:101D80000401560E8D6F040E8E6F96EF0EF00B0E43
:101D900004018F5D01E31200010E9017040103514D
:101DA00004018F5D46E150C400FD51C401FD52C4E1
:101DB00002FD53C403FD54C404FD55C405FD56C4BF
:101DC00006FD57C407FD58C408FD59C409FD5AC48F
:101DD0000AFD5BC40BFD5CC40CFD5DC40DFD5EC45F
:101DE0000EFD5FC40FFD60C410FD61C411FD62C42F
:101DF00012FD63C413FD64C414FD65C415FD66C4FF
:101E000016FD67C417FD68C418FD69C419FD6AC4CE
:101E10001AFD6BC41BFD6CC41CFD6DC41DFD6EC49E
:101E20001EFD6FC41FFD90516791E8A00AD0678125
:101E300008D08FC48CF40401000E8A6F0D0E8B6FD6
:101E400027DF040190510D011791E8B017818FC46D
:101E50009CF40401000E9A6F0D0E9B6FDFEF10F0E3
:101E60000B0E0401915D01E312009251030801E29F
:101E70001200040103510401915D47E150C400FDCB
:101E800051C401FD52C402FD53C403FD54C404FDFA
:101E900055C405FD56C406FD57C407FD58C408FDCA
:101EA00059C409FD5AC40AFD5BC40BFD5CC40CFD9A
:101EB0005DC40DFD5EC40EFD5FC40FFD60C410FD6A
:101EC00061C411FD62C412FD63C413FD64C414FD3A
:101ED00065C415FD66C416FD67C417FD68C418FD0A
:101EE00069C419FD6AC41AFD6BC41BFD6CC41CFDDA
:101EF0006DC41DFD6EC41EFD6FC41FFD0401000EE8
:101F0000886F0D0E896F95DE08D091C48CF40401A2
:101F1000000E8A6F0D0E8B6FBBDE0401925108E03C
:101F200092C4BBF60DCDBAF666EC4BF0000912E098
:101F300092C40EFD91C49CF40401000E9A6F0D0E24
:101F400092D90401915D06E192C45EF492C4FDF55C
:101F50000501FC8112000B0E0401935D01E31200E8
:101F600095C431F696C432F636EC30F0000901E142
:101F7000120004019451420A10E0090A0EE0060A18
:101F80000CE00C0A01E01200800E955D010E9659DE
:101F900004E2800E956F010E966F04010351040157
:101FA000935D47E150C400FD51C401FD52C402FDE0
:101FB00053C403FD54C404FD55C405FD56C406FDB9
:101FC00057C407FD58C408FD59C409FD5AC40AFD89
:101FD0005BC40BFD5CC40CFD5DC40DFD5EC40EFD59
:101FE0005FC40FFD60C410FD61C411FD62C412FD29
:101FF00063C413FD64C414FD65C415FD66C416FDF9
:1020000067C417FD68C418FD69C419FD6AC41AFDC8
:102010006BC41BFD6CC41CFD6DC41DFD6EC41EFD98
:102020006FC41FFD0401000E886F0D0E896F01DE65
:1020300008D093C48CF40401000E8A6F0D0E8B6FD0
:1020400027DE040194514D0A15E0060A0EE0090A44
:1020500007E0030A13E195C411FD96C412FD0ED0EA
:1020600095C40FFD96C410FD09D095C413FD96C408
:1020700014FD04D095C418FD96C419FD93C49CF4B6
:102080000401000E9A6F0D0EEED80401935D1DE160
:1020900094514D0A16E0060A0FE0090A08E0030A07
:1020A00001E0120095C461F496C462F4120095C474
:1020B0005FF496C460F4120095C463F496C464F4AB
:1020C000120095C468F496C469F4120001D9EF5067
:1020D000146E156A200E145C000E155801E2000CF7
:1020E000F7D8010EEB50030801E0000CF1D8020E06
:1020F000EB50A40801E0000CEBD8030EEB500401F8
:10210000995D01E0000C0601200EA66F97C4A4F6AD
:1021100098C4A5F6DEEC4AF0000901E0000C010CC1
:1021200050C400FD51C401FD52C402FD53C403FD5F
:1021300054C404FD55C405FD56C406FD57C407FD2F
:1021400058C408FD59C409FD5AC40AFD5BC40BFDFF
:102150005CC40CFD5DC40DFD5EC40EFD5FC40FFDCF
:1021600060C410FD61C411FD62C412FD63C413FD9F
:1021700064C414FD65C415FD66C416FD67C417FD6F
:1021800068C418FD69C419FD6AC41AFD6BC41BFD3F
:102190006CC41CFD6DC41DFD6EC41EFD6FC41FFD0F
:1021A0000401000E886F0D0E896F43DD03C49CF49B
:1021B0000401000E9A6F0D0E9B6FDFEF10F00B0EF7
:1021C00004019C5D01E3120006011F0EA66F9AC474
:1021D000A4F69BC4A5F6DEEC4AF0FF0DF350E66EC4
:1021E0009AC4E9FF9BC4EAFF1F0E1DD8E552E750D1
:1021F000EF6E0501200EFA6F9AC4F8F59BC4F9F54D
:1022000004019C51200DF3CFF6F5F4CFF7F5800EC5
:102210000501F627000EF72344EF3FF07CC4E9FFE9
:102220007DC4EAFF1200E926000EEA22120084C4EF
:10223000E9FF85C4EAFF0E0EEB50120070C4E9FFFF
:1022400071C4EAFF12001450030BF36EFC0EEF147E
:10225000F310EF6E12000D0EEB500601BA6F66EC34
:102260004BF0000912009B6FAADF0401035112001A
:1022700074C4E9FF75C4EAFF0E0EEB5012000501AD
:10228000F127000EF2231FEF3FF0030B0601BB6F97
:102290000DCDBAF666EC4BF000091200200DF3CF1D
:1022A000F1F5F4CFF2F5120072C4E9FF73C4EAFF4E
:1022B000120088C4E9FF89C4EAFF12008AC4E9FF5A
:1022C0008BC4EAFF12008DC4E9FF8EC4EAFF12003E
:1022D00097C4E9FF98C4EAFF12000D0EEB50040109
:1022E000816FBEEF0DF00501EC27000EED23F0EF3E
:1022F0003EF094DF060E13EF11F0060E94DFEF5060
:10230000030B1200060E8FDF23EF11F0EE6E010EAD
:10231000ED6E0EEF11F092DF7DEF11F0EF6E0EEF2C
:0223200011F0BA
:0E2322008F50020B01E0010EA2EC15F0EF50FF
:10233000800B01E0010E145C01E0000C17EC49F089
:10234000A2EC15F0EF50400B01E0010E145C01E02F
:10235000000CFFEC4AF0A2EC15F0010EEB50145CFF
:1023600001E0000CD2EC45F00D01026F6DC3E9FFF6
:102370006EC3EAFF020EEB50025D01E0000C010C9F
:10238000060EE66EE66AE6686FC3E6FF70C3E6FF18
:1023900020EC4BF0050EE15E12000D01086B050EFE
:1023A000085D19E20851DFDB13E10829096F060E09
:1023B000095D0EE20951D7DB09E0095157DB60DB0B
:1023C000085154DB6ADB095175DB02D0092BEFD7CA
:1023D0000D01082BE4D712000D010A6B060E0A5DF1
:1023E00056E20A51C0DB50E00A51C8DB0301715DBF
:1023F0004BE10A0E6C5D48E26CC37BF30301300EC7
:10240000796F030E7A6F0D010A51060DF3CF77F342
:10241000F4CF78F30C0E03017727030E782349D904
:10242000146E156AFF0E14182FE1000E15182CE11A
:10243000A9DBEF500501196F1A6B03016C510501FF
:10244000176F186B0501BD0E92DB020EE926000E18
:10245000EA22EF500501196F1A6B94DBEE52EF5030
:102460000501176F186B0501BE0E81DB09DB030147
:102470006C51060DF3CFE9FFF4CFEAFF300EE926E9
:10248000030EEA220ADB6C2B0D010A2BA7D71200E0
:102490000B0E0301725D01E312007351030801E2A8
:1024A000120072C3A7F5D7EC31F0F3CF02FDF4CFE1
:1024B00003FD0D01006B016B01510319E8AE02D061
:1024C000033504D00251005D035101593BE2046B16
:1024D00000CD56F601CD57F672C355F61FEC40F00D
:1024E000F3CF05FDF4CF06FDF3CF5BF6F4CF5CF63A
:1024F00058EC40F00D01076B060E075D15E2075121
:1025000032DB0FE00301735106E00D01075136DBAA
:102510000301735D06E10D010751CCDA0D01010ED7
:10252000046F0D01072BE8D7045107E036DF05CD16
:102530005DF606CD5EF666EC40F00D01002B000E58
:102540000123BAD7120074C377F675C378F69FECEF
:1025500048F0F3CF74F3F4CF75F3F3CF63F6F4CF11
:1025600064F647EC3AF00D01006F74C3AEF575C325
:10257000AFF548EC32F0F3CF01FDF4CF02FD0D01D1
:10258000056B066BF4340DE201510208000E025592
:1025900008E201CD05FD02CD06FD020E055F000E2D
:1025A000065B00CDA7F5D7EC31F0F3CF07FDF4CFF4
:1025B00008FD0D01010E075F000E085B020E156A93
:1025C0000125146E0251152208511518E8AE02D0EB
:1025D000153404D01450075D1550085906E2020E58
:1025E0000125076F000E0221086F010E0125036F00
:1025F000000E0221046F02510619E8AE02D0063522
:1026000004D00551015D0651025915E30501005141
:1026100009E001CD19F502CD1AF501CDB7F502CDCE
:10262000B8F568DA0D0101CD59F602CD5AF6010769
:10263000000E025B7FDA0D0108510419E8AE02D0EA
:10264000043504D00351075D0451085915E3050111
:10265000005109E003CD19F504CD1AF503CDB7F506
:1026600004CDB8F547DA0D0103CD59F604CD5AF67D
:10267000032B000E04235EDA0A0E03016C5D01E3F6
:1026800012000D0102510619E8AE02D0063504D041
:102690000551015D06510259AEE208510419E8AE38
:1026A00002D0043504D00351075D04510859A3E258
:1026B00012000D01096B03017B510D01095D16E24A
:1026C000030179C380F37AC381F3060E7927000EE4
:1026D0007A2377C37EF378C37FF38CD8000903E0B5
:1026E0000D01095112000D01092BE5D7FF0C11DA7C
:1026F000EF6A1CEC48F0146E0CDAE850030BF36E32
:10270000FC0EEF14F310EF6E04DA8F50020B02E0B0
:10271000EF8E01D0EF9E17EC49F0146EFAD9E85015
:10272000010BF36EF346F346F346F346F346F346E6
:10273000BF0EEF14F310EF6ED2EC45F0E66EE9D960
:10274000020EE926000EEA22E552E750EF6EFFEC9A
:102750004AF0E66EDED9EE52E552E750EF6ED9D977
:10276000030E2BC6EBFF040E2CC6EBFF1200030179
:10277000066B06810693069D069F076B086B096B27
:10278000010E0A6F12000301060E7B6F03010C0E8F
:10279000796F030E7A6F0301000E776F030E786F67
:1027A00088DF0D01056FE850146E156AFF0E1418CE
:1027B00002E1155003E005517DD9E5D7EEDD0D01AD
:1027C000050E056F0551000808E205054FD958D9D7
:1027D00005514CD962D90507F5D700C30CF301C3E5
:1027E0000DF302C30EF303C30FF304C310F305C3C9
:1027F00011F31200B3D9EF50ABD9EF50145C01E0E4
:10280000000CACD9010EEB50A3D9010EEB50145CB7
:1028100001E0000CA3D9020EEB509AD9020EEB5046
:10282000145C01E0000C010C84C3A7F621EC48F015
:10283000000901E1000C03018251831101E1000C48
:1028400082C354F483C355F485C38CF386C38DF3DC
:1028500084C38BF382C389F383C38AF384D80D01C5
:102860000B6F060E0B5D2DE20B517DD92AE00B514B
:1028700085D90301845D25E10D010B51F7D84ED9AF
:1028800020E00D010B51F2D8EECF56F4EECF57F405
:10289000EECF58F4EECF59F4EECF5AF4EFCF5BF40D
:1028A000050100510DE0520E0501116F126BE3ECB2
:1028B00022F00601560E026F040E036FA4EC34F0F2
:1028C000010C000C0301000E7C6F030E7D6F0FDF07
:1028D00003010051030B0601A76F21EC48F000092A
:1028E00041E087C363F688C364F647EC3AF00D0114
:1028F000006F87C3AEF588C3AFF548EC32F0F3CF75
:1029000001FDF4CF02FDF3CF56F6F4CF57F600CD1C
:1029100055F61FEC40F0F3CF03FDF4CF04FDF3CFE9
:102920000DF6F4CF0EF601CD0BF602CD0CF687C3F3
:1029300009F688C30AF638EC35F003CD5BF604CD12
:102940005CF658EC40F01FDF0501240E756F0501A1
:102950000C0E736F030E746F03CD71F504CD72F519
:10296000E9EC28F0120089C363F68AC364F647ECE9
:102970003AF00D01016F89C3AEF58AC3AFF548EC9B
:1029800032F0F3CF02FDF4CF03FD010E0D01F3246D
:10299000046F000EF420056F01CDA7F5D7EC31F0E0
:1029A000F3CF06FDF4CF07FD0D01800E031509E1FD
:1029B00002CD08FD03CD09FD0207000E035B86D89A
:1029C00022E305510719E8AE02D0073504D00651BD
:1029D000045D0751055909E204CD08FD05CD09FD47
:1029E000042B000E052372D80EE3800E0315DCE0E5
:1029F00005510719E8AE02D0073504D00651045D31
:102A000007510559D1E308CDB7F509CDB8F501CD8A
:102A1000B6F5A8EC32F0F3CF19F5F4CF1AF50D01A5
:102A200000510501176F186B510E0501156F166BDC
:102A300062EC23F00D01005112000D010A6B060E2D
:102A40000A5D13E20A518FD80DE00A510FD866D8FB
:102A500009E00D010A5192D803018E5D03E10D01D9
:102A60000A5112000D010A2BEAD7FF0C060DF3CF15
:102A7000E9FFF4CFEAFF0C0EE926030EEA2212006A
:102A8000EECF14F0EECF15F0EECF16F0EECF17F03C
:102A9000EECF18F0EFCF19F0120014C0EEFF15C002
:102AA000EEFF16C0EEFF17C0EEFF18C0EEFF19C014
:102AB000EEFF1200060DF3CF6FF3F4CF70F30C0EA0
:102AC00003016F27030E7023C0EF11F008CD59F6F4
:102AD00009CD5AF601CD58F64BEC40F08CC38FF37C
:102AE0008DC390F38BC38EF3A8DF0D01006F060E2C
:102AF000005D120000CDB6F5A8EC32F0F3CF17F56B
:102B0000F4CF18F505015A0E156F020E166F62EF1D
:102B100023F07CC3E9FF7DC3EAFF1200030EE92620
:102B2000000EEA22EECF31F6EDCF32F636EC30F081
:102B30000009120000CD58F64BEC40F076C371F35B
:102B4000ECEF11F0146E6DC3E9FF6EC3EAFF1200E3
:102B5000146E80C3E9FF81C3EAFF12007EC3E9FF60
:102B60007FC3EAFF120082DFEF50FF081200156FEB
:102B7000020E166F62EC23F0C2EF15F077DFEF5014
:0C2B8000030B12000D010A5136EF15F096
:042B8C0077C5E9FF21
:102B900078C5EAFFEF50570A01E18ED0010A01E142
:102BA00085D0020A01E17CD0070A74E0010A6CE0DA
:102BB000020A64E01D0A5CE0010A54E0050A4CE0E8
:102BC0000E0A42E0010A3AE0030A32E0010A26E076
:102BD000070A15E0010A0DE0030A05E07A0A75E12B
:102BE00049EC33F072D077C579F578C57AF573D8AA
:102BF0006CD077C57BF578C57CF5DCD866D022DB58
:102C0000540805E145DB03E139EC06F05ED077C5F9
:102C1000A9F378C5AAF319EC06F057D013DB4D08D9
:102C200054E177C5ABF378C5ACF33FEC06F04DD07B
:102C300077C57DF578C57EF5DED847D077C57FF5B9
:102C400078C580F50DD941D0FDDA4F083EE120DB93
:102C50003CE12AEC07F039D0F5DA3B0836E138ECF4
:102C600007F033D077C581F578C582F548D92DD0E6
:102C700077C583F578C584F557D927D077C585F50D
:102C800078C586F577D921D077C587F578C588F5D9
:102C900097D91BD077C589F578C58AF5AED915D0F7
:102CA00077C58BF578C58CF5DDD90FD077C58DF557
:102CB00078C58EF567DA09D0C5DA4B0806E177C525
:102CC000EBF378C5ECF304EC0AF00501765100084B
:102CD00001E276071200010E05019CDA550A5CE05C
:102CE000010A4DE0040A45E01E0A3DE0030A2EE019
:102CF000060A1FE0030A14E00E0A09E0030A01E0D5
:102D0000120079C591F37AC592F31DEF04F0D2DA7F
:102D100054084FE179C593F37AC594F357EF04F063
:102D2000C9DA340846E179C595F37AC596F38DEF93
:102D300004F0C0DA49083DE1030E6CDA500839E1CD
:102D400079C599F37AC59AF3D6EF04F0B3DA50084F
:102D500030E1030E5FDA49082CE179C59BF37AC5AF
:102D60009CF3EFEF04F079C59DF37AC59EF313EF62
:102D700005F079C59FF37AC5A0F348EF05F09ADA1C
:102D8000540817E1030E46DA4E0813E179C5A1F3A2
:102D90007AC5A2F37EEF05F08DDA58080AE1030E3A
:102DA00039DA460806E1040E35DA3B0802E19DEC0B
:102DB00005F01200010E05016FDA590A11E00B0A45
:102DC00009E01C0A01E012007BC5A3F37CC5A4F353
:102DD0009FEF05F07BC5A5F37CC5A6F3C7EF05F013
:102DE000020E5ADA500806E17BC5A7F37CC5A8F3AA
:102DF000FCEC05F01200010E050128DA570A29E063
:102E0000050A21E01F0A19E0080A01E01200020E7B
:102E10001DDA490824E1030E19DA4E0820E1040EF8
:102E200015DA49081CE1050E11DA540818E1060EFE
:102E30000DDA3B0814E14DEF06F07DC5ADF37EC51C
:102E4000AEF35AEF06F07DC5E1F47EC5E2F4ACEFD7
:102E500024F07DC5E3F47EC5E4F4FBEC24F012001D
:102E6000010E0501E5D9570A3AE0030A33E0180AD2
:102E70001FE00A0A10E0030A08E0040A39E17FC5EE
:102E8000B1F380C5B2F3A0EF06F025DA3B0836E1D6
:102E9000020E766F12001FDA4D0830E1030EC8D91A
:102EA00054082CE1040EC4D93B0828E1D2EF06F007
:102EB00012DA540A09E01D0A01E012007FC5B3F3DB
:102EC00080C5B4F3DDEF06F07FC5B5F380C5B6F37A
:102ED000F5EF06F000DA3B0811E1F4EF42F0FBD920
:102EE00053080CE17FC5B7F380C5B8F30DEF07F0C9
:102EF0007FC5AFF380C5B0F385EC06F01200010E7C
:102F00000501BFD950080AE1020EBBD9460806E107
:102F1000030EB7D93B0802E188EF42F081C5B9F34F
:102F200082C5BAF346EF07F0010E0501BCD9540A79
:102F300009E0100A01E0120083C5BBF384C5BCF3AD
:102F400063EF07F0020EAFD94D0A08E00C0A0CE15E
:102F500083C5BFF384C5C0F38EEF07F083C5C1F30B
:102F600084C5C2F3ABEF07F083C5BDF384C5BEF3E0
:102F700086EF07F0010E05017ED9EF50530A0EE0EF
:102F8000030A01E01200030E76D9EF503B0817E167
:102F9000020E71D9EFCFA3F6ABEF42F0020E6BD960
:102FA000EF50490806E185C5C5F386C5C6F3E1EFD4
:102FB00007F085C5C3F386C5C4F3C8EC07F012005B
:102FC000010E05014AD9560A11E0050A01E0120076
:102FD000020E43D9540810E1040E3FD93B080CE11E
:102FE00087C5C7F388C5C8F3FEEF07F0020E35D9D1
:102FF0003B0802E111EC08F01200010E050134D982
:10300000540A29E01A0A21E0030A19E0010A11E032
:10301000050A01E01200020E27D9440822E1030E3E
:1030200023D945081EE189C5C9F38AC5CAF321EF32
:1030300008F089C5CBF38AC5CCF33CEF08F089C50D
:10304000CDF38AC5CEF359EF08F0020E0DD93B0837
:1030500008E165EF39F089C5CFF38AC5D0F37FEC7D
:1030600008F01200010E050128D9560A01E183D0AB
:10307000050A01E17BD0010A70E0020A48E0190A62
:1030800034E00C0A2CE0060A10E0020A05E07A0A95
:1030900001E01200F4EF42F0D2D8500872E18BC583
:1030A000D1F38CC5D2F311EF09F0C9D8560A11E05B
:1030B000040A09E0140A01E012008BC5D5F38CC59F
:1030C000D6F354EF09F08BC5D7F38CC5D8F361EF75
:1030D00009F08BC5D9F38CC5DAF36EEF09F08BC517
:1030E000D3F38CC5D4F31EEF09F0A9D8500A09E038
:1030F000110A01E012008BC5DBF38CC5DCF370EF25
:1031000009F08BC5DDF38CC5DEF37DEF09F097D8B0
:10311000560A1DE0060A15E0120A0DE0030A05E052
:103120007A0A01E012008AEF09F08BC5DFF38CC543
:10313000E0F397EF09F08BC5E1F38CC5E2F3A4EF60
:1031400009F08BC5E3F38CC5E4F3C1EF09F08BC53F
:10315000E5F38CC5E6F3CEEF09F071D8490811E12B
:103160008BC5E7F38CC5E8F3DBEF09F068D83B08C3
:1031700008E1ADEF44F08BC5E9F38CC5EAF3E6EC6A
:1031800009F01200010E05014CD8530A21E0010A92
:1031900011E0140A01E01200020E43D8570839E189
:1031A000030E3FD8440835E1040E3BD83B0831E11B
:1031B00075EF2DF0020E35D846082BE1030E31D8FD
:1031C0004C0827E1040E2DD83B0823E187EF2DF0B2
:1031D000020E27D857081DE1030E23D8520819E123
:1031E000040E1FD8420A0BE0790A01E01200E3EC5A
:1031F0002FF0F3CF96F6F4CF97F6DCEF48F0050EFC
:1032000010D83B0806E12BC698F62CC699F6E5ECDB
:1032100048F01200EA6A7925E96E7A51EA22EF5005
:103220001200EA6A8D25E96E8E51EA22EF501200F3
:10323000EA6A7F25E96E8051EA22EF501200020E01
:103240005DEF19F0010E050164EF19F0EA6A7D25C2
:10325000E96E7E51EA22EF501200EA6A8725E96E94
:103260008851EA22EF501200EA6A8925E96E8A51F4
:10327000EA22EF501200EA6A8525E96E8651EA22B9
:103280001200EA6A8125E96E8251EA22EF501200AB
:10329000020E1AD83B081200EA6A7B25E96E7C51BF
:1032A000EA22EF501200EA6A8325E96E8451EA228D
:1032B000EF501200020E0AEF19F0EA6A8B25E96E50
:1032C0008C51EA22EF501200EA6A7725E96E7851B4
:0C32D000EA22EF501200020E18EF19F075
:0432DC0006018D5109
:1032E000040B03E18D51080B14E08D958D975DDA89
:1032F000820E6BDA0EE149DA0401500E706F040E93
:10330000716F42EC0BF0000904E05BDA02E00501AA
:10331000FC8B12000501FCA12CD0FC9146DA8C0E2E
:1033200054DA27E169DA0501FD5D23E0FDC5BBF64E
:103330005DC4BAF666EC4BF000090FE026DA050131
:10334000FD510401030BF36EFC0E5615F310566F7E
:1033500038DA0FE00501FC8B120004015D51050114
:10336000196F1A6B0501FD510501176F186B8F0E50
:1033700012DA1200C2EC1CF0000907E03FC6FEF5AD
:1033800040C6FFF50501FC8702D069EC35F0050168
:10339000FCA722D0FE51FF111FE0FEC563F6FFC55A
:1033A00064F647EC3AF00D01206FE8CF40F47FEC73
:1033B0001EF0000911E0FEC519F5FFC51AF50D0153
:1033C00020510501176F186BA20EE5D90501E66BB8
:1033D000F8D902E00501FC8B120006018DA11BD07B
:1033E0008D9106017397E1D90401F66BF76B26EC1A
:1033F0001DF0000910E108C400FD790ED1D90501C6
:10340000E66B6AEC1EF0420E0D01005D04E1D9D9B5
:1034100002E00501FC8B1200D4D924E0C2EC1CF0C0
:10342000000920E00401545106013F1904E10401A0
:1034300055510601401916E054C4B9F555C4BAF502
:10344000DBEC32F000090EE051EC20F0000909E15C
:103450003FC663F640C664F647EC3AF00401035DEC
:1034600001E0BAD9120006018D51100B03E18D5114
:10347000200B07E08D998D9B0501FC8996D9960E4E
:103480008FD91200AADF2ADF45DFEDDF73DF0501E8
:10349000FCB903D096D901E0BFDF0501FCA90DD02E
:1034A000B40E7ED9420E0401085D05E104014D0E03
:1034B0004A6FCDEC1FF0050109D0DCEC35F00009B6
:1034C00009E0BE0E6DD988D90501FC83FC8F060189
:1034D00073937395010E236E0501FCAB5AD0FC9BD0
:1034E000FEC519F5FFC51AF582D9BB0E54D90501E1
:1034F000FC51080B03E0FE51FF1111E1040154518E
:1035000055110DE054C4FEF555C4FFF50501FC87C7
:1035100054C419F555C41AF56AD9BC0E3CD9050135
:10352000FC51080B03E0FE51FF1111E103C466F6E4
:103530005FEC3AF0F3CFFEF5F4CFFFF50501FC8721
:10354000F3CF19F5F4CF1AF552D9BD0E24D90501E0
:10355000FC51080B1EE0FE51FF111BE02AD9FEC5ED
:1035600082F3FFC583F314EC14F0000910E0FEC5EC
:1035700054F4FFC555F4B1D8000909E1060173B34D
:1035800006D059C433F65AC434F680EC30F0050145
:10359000FC978AD80501FCA903D00601260E19D094
:1035A0008FA60CD006011C510401225D06011D519D
:1035B0000401235903E20601270E0BD086D8000927
:1035C00003E00601280E05D088D8000903E00601B3
:1035D000290E08D152EC47F0000901E01200DCECA2
:1035E00035F0000907E00501FC89FC83FC8F06012A
:1035F000350E05D00501FCA903D006013A0EF2D024
:103600000F0E236E14EC30F0000901E012008FA2BF
:103610003AD02BC6F4F42CC6F5F4D8EC1CF0000913
:1036200008E029C6F4F42AC6F5F4D8EC1CF0000929
:103630002AE12BC62DF52CC62EF51CC62BF51DC672
:103640002CF50501940E296F020E2A6FF1EC23F080
:1036500029C62DF52AC62EF51CC62BF51DC62CF540
:103660000501950E296F020E2A6FF1EC23F088EC0C
:103670003BF0000905E10601020E9F6F05EC3BF0EF
:103680000401569F120044EC30F0000903E08DD88D
:1036900006017397060173B705D0FCEC42F00009F0
:1036A00001E01200236A1200A7D8146E010E145C08
:1036B00004E35651030B030807E20401500E726F36
:1036C000040E736F6EEC0BF012001CEC48F0146EDD
:1036D00093D8145C01E0010E12000D01560E006F2C
:1036E000040E016F420E0401085D04E0040156510E
:1036F000800B05E10D01060E006F030E016F00CD7A
:103700006DF301CD6EF391EC11F0000901E0000CB6
:10371000010C0601AC51AD1101E1000C52D801E1E0
:10372000000CACC694F6ADC695F6F2EC44F02BC690
:103730002DF52CC62EF560D805012B6F2C6BCD0E08
:103740000501296F2A6BF1EC23F033D8ACC682F364
:10375000ADC683F314EC14F0000901E1000C59C468
:103760002DF55AC42EF554C42BF555C42CF5CF0EA7
:103770000501296F2A6BF1EC23F0040159515F5DBB
:103780005A51605901E2568F010C36D85E5D02E154
:1037900090EC10F012000501156F166B62EF23F02C
:1037A0000501116F126BE3EF22F00601A06BA6EF8B
:1037B0003BF02BC685F32CC686F31ED80301846F1D
:1037C0001200F2EC1EF0000912000401F66FF76B14
:1037D00026EC1DF0000912003FC6FAF040C6FBF0CF
:1037E000A9EF35F0BC6F020EBD6F1FEF43F0FC5127
:1037F0000501176F186B120004015651030B1200DC
:103800004EDAE9C419F052DAE9C407F029DA3CD2F9
:10381000EAC4F2F4EBC4F3F491D80D01006FE8CFE1
:10382000FCF4ABD9F3CF07FDF4CF08FD00CDE9F4EC
:10383000E7DFF3CF0BFDF4CF0CFD0D0107510401C1
:10384000EA190AE10D0108510401EB1905E10BCD5C
:10385000F3FF0CCDF4FF12000D0100050401FC6F15
:103860008CD9F3CF05FDF4CF06FD0D01000525DA57
:10387000F3CF09FDF4CF0AFD0BCD53F60CCD54F672
:1038800020DA07CD4FF608CD50F605CD4DF606CD22
:103890004EF6EAC44BF6EBC44CF607EF42F0200EAE
:1038A000086E096AECC40DF0EDC40EF046EC44F06D
:1038B00006C0EAF407C0EBF408EF1CF006011C5147
:1038C0000401285D06011D510401295914E228C490
:1038D00019F529C41AF51CC617F51DC618F5EEC44E
:1038E00015F5EFC416F562EC23F00601030E9F6F89
:1038F00005EC3BF0010C000C0D01136B7D0E146FF9
:103900000D011451135D18E21351145DFE0BE842D2
:103910001325156FDBD9F3CF14F0F4CF15F00401A4
:10392000F051F35CF151F45804E20D011529136FC5
:10393000E7D715CD14FDE4D7135112000D01116B1B
:103940007D0E126F0D011251115D1AE21151125DBF
:10395000FE0BE8421125136FE8CFFCF40ED9F3CF2C
:1039600014F0F4CF15F00401F251F35CF351F45864
:1039700004E20D011329116FE5D713CD12FDE2D733
:103980001151120004011A5106011C5D04011B5162
:1039900006011D5901E3010C000C0401265106012A
:1039A0001C5D0401275106011D5901E3010C000CA7
:1039B00004012C5106011C5D04012D5106011D5905
:1039C00001E2010C1C5104012A5D06011D51040194
:1039D0002B5901E2000CF4C4F8F4F5C4F9F453D8FF
:1039E000F3CF0DFDF4CF0EFDF3CFEAF4F4CFEBF4FB
:1039F0000FDFF3CF0FFDF4CF10FD06011C510D01B9
:103A0000F35C06011D510D01F45801E3010CF4C4EF
:103A10002DF5F5C42EF51CC62BF51DC62CF505019C
:103A2000600E296F010E2A6FF1EC23F00FCD19F50E
:103A300010CD1AF50DCD17F50ECD18F50501610E57
:103A4000156F010E166F62EC23F0000C0401185183
:103A500006011C5D0401195106011D5901E3010C09
:103A60000401F651F7110EE018C419F519C41AF53E
:103A70001CC617F51DC618F5F6C415F5F7C416F5DE
:103A800062EC23F0000C0401000EF85D1C0EF959E5
:103A900004E3400EF36E1F0E07D0E40EF85D030E34
:103AA000F95904E2F36AE10EF46E1200F8C41AF058
:103AB000F9C41BF01C6A1D6A166A176A6B0E186E31
:103AC000030E196E16C006F017C007F018C008F0F4
:103AD000096EF8C40BF0F9C40CF01CC00DF01DC049
:103AE0000EF0BAEC4AF006C0F3FF07C0F4FF120074
:103AF000FAC4F0F4FBC4F1F4FFDE0D01006FE6D868
:103B0000F3CF03FDF4CF04FD00CDFCF436D8F3CFA2
:103B100007FDF4CF08FD0D0103510401FA190AE174
:103B20000D0104510401FB1905E107CDF3FF08CD98
:103B3000F4FF12000D010005C0D8F3CF01FDF4CF52
:103B400002FD0D0100050401FC6F17D8F3CF05FD40
:103B5000F4CF06FD07CD53F608CD54F6B2D803CD09
:103B60004FF604CD50F601CD4DF602CD4EF6FAC417
:103B70004BF6FBC44CF607EF42F091D8FCC419F0A9
:103B800095D8FCC407F06CD8020EF626000EF7227A
:103B9000F8227AD014C4ECF415C4EDF480DEF3CF2F
:103BA00016F4F4CF17F404011851F35C1951F458CA
:103BB00004E218C416F419C417F41200FDC4F0F49A
:103BC000FEC4F1F499DE0D010A6F80D8F3CF0DFD2C
:103BD000F4CF0EFD0ACDFFF436D8F3CF11FDF4CFAC
:103BE00012FD0D010D510401FD190AE10D010E51E7
:103BF0000401FE1905E111CDF3FF12CDF4FF12000F
:103C00000D010A055AD8F3CF0BFDF4CF0CFD0D01C1
:103C10000A050401FF6F17D8F3CF0FFDF4CF10FD95
:103C200011CD53F612CD54F64CD80DCD4FF60ECD26
:103C300050F60BCD4DF60CCD4EF6FDC44BF6FEC442
:103C40004CF607EF42F02BD8FFC419F02FD8FFC471
:103C500007F006D8040EF626000EF722F82214D03C
:103C60001AC008F01BC009F064EC44F0165004249C
:103C7000F36E17500520F46E18500620F86EF4CF3E
:103C8000F7FFF3CFF6FF12000900F5CF14F008009C
:103C9000F5CF15F014C0F3FF15C0F4FF1200D40ED9
:103CA000166E550E176E000E186E12001A6A1B6AF9
:103CB000060E0C6E0D6A0E6A12000401E96F00EF29
:103CC0001CF0F3CF51F6F4CF52F61200E8CFE9F42E
:043CD00000EF1CF0F5
:0C3CD40004010851420A0CE00F0A07E04E
:103CE000180A02E0140A06E104014D0E05D0040191
:103CF000420E02D00401410E4A6FCDEF1FF00401C5
:103D00000351405D01E1000C0B0E405D01E3000C2E
:103D1000550E085D02E090EC10F040C444F406EF4C
:103D20001FF0200E1BD20401000E415D040E42590B
:103D300015E241C4ECF542C4EDF5F0EC3EF0FF08AD
:103D400008E00501F06941C4EEF542C4EFF502EC6C
:103D50003FF00401412B000E4223E5D71200020E72
:103D6000FDD1400EE66EE66ACC0EE66E000EE66E03
:103D7000040EE66E20EC4BF0050EE15E0401400EF1
:103D8000006F040E016FA30E026F330E046F190E45
:103D9000056F066B036B450E076F1E0E146F156BD8
:103DA000410E086F096B0981098D098F12005ED8D9
:103DB00003C421FD0D01206B0B0E205D07E220CD19
:103DC00003F4F2EC0DF00D01202BF6D721CD44F4D5
:103DD0001DD8040109A103D00601C28F12000601FB
:103DE000C28D120004010851410A02E00C0A01E1EF
:103DF000010C000C04014351410A06E0030A04E0EF
:103E00000F0A02E0180A01E1010C000C0401035141
:103E1000445D01E1000C0B0E445D01E3000C44C461
:103E200003F4F0EC3AF03FEC0EF0550E0401085D9F
:103E300007E10301560E7C6F040E7D6F77EC13F0E3
:103E40000401500E726F040E736F6EEC0BF065D9A7
:103E50000501E66B0601A06BA6EC3BF0C2EC1CF082
:103E6000000903E106013F6B406B010C0501400EA8
:103E7000F56F0501000EF36F040EF46F200E0501BF
:103E8000F16FF26B1FEC3FF01AD9000901E169DF15
:103E9000010E57D9F3CF18F4F4CF19F4040E51D909
:103EA000F3CF1AF4F4CF1BF4070E4BD9F3CF1CF465
:103EB000F4CF1DF4040E45D9F3CF1EF4F4CF1FF454
:103EC0003C0E3FD9F3CF20F4F4CF21F41E0E39D9A4
:103ED000F3CF22F4F4CF23F40A0E33D9F3CF24F432
:103EE000F4CF25F4050E2DD9F3CF26F4F4CF27F423
:103EF000D20E27D9F3CF28F4F4CF29F40401080E09
:103F0000EC6F070EED6F4FEC1CF0F3CF2AF4F4CFFB
:103F10002BF4FA0E16D9F3CF2CF4F4CF2DF4190E9E
:103F200010D9F3CF2FF4F4CF30F404012E6BCAEC88
:103F30001DF007C44FF446EF20F00401010E455D6B
:103F4000000E465903E2010E456F466BDC0ED88029
:103F50004555050E465504E2DC0E456F050E466FCD
:103F600045C414F446C415F4CAEC1DF08DEF20F0DE
:103F7000040147510991E8B009818DEF20F0040157
:103F80004851099DE8B0098D8DEF20F00401495199
:103F9000099FE8B0098F8DEF20F0040108514A5DB8
:103FA00001E1000C4AC443F425DF000901E1000CE3
:103FB0000601BC6BBD6B1FEC43F04AC408F4ADD8DE
:103FC0000AEC3AF0010C04014B51099BE8B0098B53
:103FD0008DEF20F004014C515A0A54E0020A4DE0E2
:103FE0000F0A46E0040A3FE0070A38E0060A31E01B
:103FF0001E0A2AE00A0A23E0030A1CE0010A15E06F
:10400000070A0EE0010A07E0030A3EE14DC422F46C
:104010004EC423F439D04DC42AF44EC42BF434D00A
:104020004DC41EF44EC41FF42FD04DC424F44EC40E
:1040300025F42AD04DC420F44EC421F425D04DC41B
:104040001AF44EC41BF420D04DC426F44EC427F4F9
:104050001BD04DC428F44EC429F416D04DC41CF412
:104060004EC41DF411D04DC42FF44EC430F40CD006
:104070004DC42CF44EC42DF407D04DC418F44EC4D6
:1040800019F402D04DC42EF48DEF20F00401075135
:10409000450A03E00C0A01E012004FC407F48DEF5B
:1040A00020F0040109AD04D0410E085D01E1010CCE
:1040B00009AF04D04D0E085D01E1010C000C0401B4
:1040C0000051146E156A400E145C000E155801E282
:1040D000000CA30E025D01E0000C04C4B2F691ECEA
:1040E0004AF0000901E1000C0B0E0401035D01E33D
:1040F000000C450E075D04E0490E075D01E0000C71
:1041000008C443F477DE000901E1000C0601400E0B
:104110001DD8000901E0000C010C06013F0E16D865
:10412000FF0DF3CF3FF40501400EFA6F0501000EBD
:10413000F86F040EF96F200E0501F66FF76B44EF70
:104140003FF00401EC6FED6B4FEF1CF0A66F060122
:10415000000EA46F040EA56FDEEF4AF00401416F5C
:06416000426B93EF1EF01C
:0A4166000B0E06010F5D01E31200CD
:10417000310EE76E1019E8AE02D0E73402D0E750F6
:10418000105D01E21200330EE76E1019E8AE02D0A6
:10419000103503D0E750D880105501E21200CBD97A
:1041A000450EE2D90FC607FF43EC33F010C68CF67C
:1041B000C3EC46F0030E060110150401876F0FC60D
:1041C00086F410EC0EF0BED10B0E0601115D07E275
:1041D00011C67FF471EC0DF00601126F01D81200C8
:1041E000AAD9450EC1D906011251010BB6D9020B4D
:1041F00001E0010EB2D9040B01E0010EA3D10B0EB8
:104200000601135D01E31200040103510601135D71
:1042100041E150C420FD51C421FD52C422FD53C4CC
:1042200023FD54C424FD55C425FD56C426FD57C4A2
:1042300027FD58C428FD59C429FD5AC42AFD5BC472
:104240002BFD5CC42CFD5DC42DFD5EC42EFD5FC442
:104250002FFD60C430FD61C431FD62C432FD63C412
:1042600033FD64C434FD65C435FD66C436FD67C4E2
:1042700037FD68C438FD69C439FD6AC43AFD6BC4B2
:104280003BFD6CC43CFD6DC43DFD6EC43EFD6FC482
:104290003FFD09D013C68CF40401200E8A6F0D0E69
:1042A0008B6F48EC0EF047D9460E52D913C607FF64
:1042B00043EC33F00D013751010B44D10B0E0601D5
:1042C000145D01E31200040103510601145D41E194
:1042D00050C400FD51C401FD52C402FD53C403FD8E
:1042E00054C404FD55C405FD56C406FD57C407FD5E
:1042F00058C408FD59C409FD5AC40AFD5BC40BFD2E
:104300005CC40CFD5DC40DFD5EC40EFD5FC40FFDFD
:1043100060C410FD61C411FD62C412FD63C413FDCD
:1043200064C414FD65C415FD66C416FD67C417FD9D
:1043300068C418FD69C419FD6AC41AFD6BC41BFD6D
:104340006CC41CFD6DC41DFD6EC41EFD6FC41FFD3D
:1043500009D014C68CF40401000E8A6F0D0E8B6F09
:1043600048EC0EF001EC23F00601540EFDD80601D6
:10437000500EFAD80601420EF7D84CEC33F003CDBC
:1043800067F695EC3AF004CD79F605CD7AF6C4ECF3
:1043900048F00601060E026F0D0E036FA4EC34F018
:1043A0000DCD12F61DDF0ECD17F603CD16F613D880
:1043B00003CD13F6FFEF20F00B0E0601155D01E3B0
:1043C000120015C683F4D3EC0DF00601176F15C665
:1043D00016F6EBEF21F0AFD8500EC6D816C607FF81
:1043E00043EC33F0300E060117110601BDD849EF3A
:1043F00033F001EC23F00B0E0601185D01E312000F
:10440000040103510601185D41E150C400FD51C48F
:1044100001FD52C402FD53C403FD54C404FD55C440
:1044200005FD56C406FD57C407FD58C408FD59C410
:1044300009FD5AC40AFD5BC40BFD5CC40CFD5DC4E0
:104440000DFD5EC40EFD5FC40FFD60C410FD61C4B0
:1044500011FD62C412FD63C413FD64C414FD65C480
:1044600015FD66C416FD67C417FD68C418FD69C450
:1044700019FD6AC41AFD6BC41BFD6CC41CFD6DC420
:104480001DFD6EC41EFD6FC41FFD09D018C68CF43F
:104490000401000E8A6F0D0E8B6F48EC0EF00601C2
:1044A0001951420A0FE0030A08E00A0A01E012006B
:1044B00013CD20FD14CD21FD09D011CD20FD12CD4D
:1044C00021FD04D00FCD20FD10CD21FD0601530E9E
:1044D0003FD818C607FF43EC33F019C68CF6C3EC7F
:1044E00046F020CD10FF21CD11FFC4EC33F049EF91
:1044F00033F00501005103E01AC614F6DFDE1200A6
:104500000501005103E01BC615F656DF1200050138
:10451000005106E006014B0E196F03C418F669DF5F
:1045200012000501005106E00601410E196F03C497
:1045300018F65FDF120001EC23F00601410E14D8DB
:10454000060112000F010A6F6DEC33F049EF33F0F2
:104550000BD80601540EB4EF22F00F010A6F6DEC78
:0E45600033F00601125112008C6FC3EF46F0CB
:02456E0049D82A
:1045700009C500F51200050100AD24D042D84FEC6A
:1045800033F00601460ED9D94D0ED7D9530E8C6F94
:10459000C3EC46F00AC50CFF0BC50DFFB5EC33F0BC
:1045A0000CC50CFF0DC50DFFB5EC33F005010E5128
:1045B0000F010C6F0D6BB5EC33F00FC50CFF10C580
:1045C0000DFFB7D91200050100510EE0115101197C
:1045D00006E11251021903E1A3D901E2A6D111C5E6
:1045E00013F512C514F501D812000BD813C501F547
:1045F00014C502F58ED913C50CFF14C50DFF99EF34
:1046000024F00501000ED8800355000E045514E275
:104610000601540E92D9440E90D9520E8C6FC3EC01
:1046200046F001C50CFF02C50DFFB5EC33F003C524
:104630000CFF04C50DFF7DD90501036B046B016BF5
:10464000026B12000501005101E112002350146EAB
:10465000156A235001191BE11550021918E10501D3
:10466000D351166E176A16500501051910E117503F
:1046700006190DE10501D4510501071908E10501ED
:10468000D5510501081903E14BD901E24ED1B9DF3B
:1046900023500501016F026B0501D3510501056F20
:1046A000066B0501D4510501071904E10501D55137
:1046B0000501081902E0000E01D0010E4FEC33F0A5
:1046C000ADEF44F0050100AB22D01551011912E104
:1046D000165102190FE1175105190CE1185106196D
:1046E00009E11951071906E11A51081903E118D90E
:1046F00001E21BD119C51FF51AC520F517C51DF517
:1047000018C51EF515C51BF516C51CF501D81200F8
:1047100078DF1BC501F51CC502F51DC505F51EC5D5
:1047200006F51FC507F520C508F5F3D81BC50CFF16
:104730001CC50DFFB5EC33F01DC50CFF1EC50DFFEC
:10474000B5EC33F01FC50CFF20C50DFF99EF24F029
:10475000050100AB24D00151211918E102512219A1
:1047600015E12351146E156A145005190FE1155007
:1047700006190CE12451166E176A1650071906E146
:104780001750081903E1CCD801E2CFD024C528F591
:1047900023C527F521C525F522C526F501D8120028
:1047A000050100AB1DD02DDF25C501F526C502F59D
:1047B00005012751056F066B2851076F086BA9D8B3
:1047C00025C50CFF26C50DFFB5EC33F027C50BFF43
:1047D000B0EC33F028C50BFFB0EC33F049EC33F00C
:1047E0001200050100AB22D02951011912E12A5112
:1047F00002190FE12B5105190CE12C51061909E1A1
:104800002D51071906E12E51081903E189D801E25B
:104810008CD02DC533F52EC534F52BC531F52CC5FF
:1048200032F529C52FF52AC530F501D8120005014A
:1048300000AB22D0E6DE2FC501F530C502F531C54B
:1048400005F532C506F533C507F534C508F561D859
:104850002FC50CFF30C50DFFB5EC33F031C50CFF93
:1048600032C50DFFB5EC33F033C510FF34C511FF71
:10487000C4EC33F049EC33F01200050100AB22D058
:104880003551011912E1365102190FE1375105195D
:104890000CE13851061909E13951071906E13A517D
:1048A000081903E13DD801E240D039C53FF53AC5CA
:1048B00040F537C53DF538C53EF535C53BF536C540
:1048C0003CF501D81200050100AB22D09ADE3BC5B1
:1048D00001F53CC502F53DC505F53EC506F53FC5EC
:1048E00007F540C508F515D83BC50CFF3CC50DFFC5
:1048F000B5EC33F03DC510FF3EC511FFC4EC33F0FD
:104900003FC510FF40C511FFC4EC33F049EC33F054
:1049100012000601540E11D8500E8C6FC3EF46F0F2
:10492000E70E035D030E04591200032B000E04234F
:104930001200B5EC33F049EF33F08C6FC3EC46F066
:04494000060112005A
:0C494400F0D8FF0DF3CFE0F4120069D9A9
:10495000FF0DF3CFE0F4120085D906D901E1000C78
:1049600088D902D901E1000C8BD9FED801E1000CF5
:1049700004019F5101E1000C9F51400801E2000C2D
:1049800086D9F2D801E1000C5FD9E02501E0000CE6
:104990000B0E3BD9EF503B0801E0000C020E35D95D
:1049A000EF50500804E1FDD800090BE1000C020EA5
:1049B0002CD9EF50530804E101D9000902E1000CA1
:1049C000000C6CD9520E8C6FC3EC46F0020E040141
:1049D0001CD96BD90D01006B04019F510D01005DC5
:1049E00005E2005136D90D01002BF6D7D1D8146E4F
:1049F0002BD914241FD136D90401AFD801E1000C02
:104A000038D90401AAD801E1000C3AD90401A5D88B
:104A100001E1000C04019F5101E1000C9F5140088D
:104A200001E2000C0D01006B04019F510D01005DBE
:104A300013E200510501A36FA46BA00EA327040E7F
:104A4000A423090E0D0100250025040186D801E1EB
:104A5000000C0D01002BE8D71AD904019F259F25D2
:104A60007CD801E1000C94D8146EEED8E025142413
:104A700001E0000C0B0E9F259F25CDD8EF503B0881
:104A800001E0000C020EC7D8EF50500804E1A3D893
:104A900000090BE1000C020EBED8EF50530804E1F0
:104AA000A7D8000902E1000C000CF8D8570E8C6F53
:104AB000C3EC46F0020E0401AED8F7D8C5D8BAD080
:104AC00032D80401E02501E0000C010CAAD8040151
:104AD000E02501E0000C010C04019F5101E1000CF4
:104AE0009F51400801E2000C010CBCEF25F0FDDFF6
:104AF0000D01006B04019F510D01005D05E20051A5
:104B0000A8D80D01002BF6D722DFE0C408FF57EF2D
:104B100033F0EBDF17DFE0C408FF57EF33F0D1EFDE
:104B200025F0DEEF25F024EF26F0C8EF25F0D4DFE6
:104B3000000901E1000CC4DF000901E1000C010CD7
:104B4000CBDF000901E1000CC1DF000901E1000C2D
:104B5000010CEBEF25F0F8EF25F0E3250501A16F3F
:104B6000000E0401E421A7D00401E1250501A16F95
:104B7000000E0401E2219FD09EC408FF57EC33F0E1
:104B80009DC408FF57EC33F09FC408FF57EF33F084
:104B90009FC4A6F60601A00EA46F040EA56FDEEF5B
:104BA0004AF09FC4F5F50501A00EF36F040EF46FF3
:104BB0009DC4F1F59EC4F2F51FEF3FF09FC46FF561
:104BC0000501A00E6D6F040E6E6F9DC46BF59EC443
:104BD0006CF585EF28F09FC4FAF50501A00EF86F7B
:104BE000040EF96F9DC4F6F59EC4F7F544EF3FF04F
:104BF0009FC475F50501A00E736F040E746F9DC4FC
:104C000071F59EC472F5E9EF28F0EA6AE125E96ED4
:104C1000E251EA221200EA6AE325E96EE451EA224F
:104C2000120083DF146EE66E7EDFE552E7CF14F0EC
:104C300014241200FF0DF3CFE0F4F3CF08FF57EC7C
:104C400033F049EC33F0010C04019E519D259F2562
:104C50001200EA6AA00FE96E040EEA22EFCF08FF05
:104C600057EF33F005019E0EA36F040EA46F030EE1
:104C7000120005019D0EA36F040EA46F050E120015
:104C800005019F0EA36F040EA46F070E120005010D
:104C9000E00EA36F040EA46F090E12000601450E6C
:104CA0008C6FC3EC46F006011200EFCF8CF6C3EC1C
:104CB00046F0BCEF25F00501A26F5AEC2AF000097E
:024CC0001200E0
:0E4CC2000501FCA31AD0060129510401615D11
:104CD00006012A510401625911E361C439F562C425
:104CE0003AF529C637F52AC638F50501920E356F13
:104CF000130E366F3DEC24F00F0E01D0060E236E1E
:104D0000120052EC47F0000901E012000601B40E57
:104D1000BC6F0F0EBD6F1FEC43F0000901E01200E5
:104D20000401BE0EEE6F0F0EEF6F5EEC1CF000097B
:104D300003E00F0E236E1200060173B30DD00601BF
:104D4000B96B77EC49F0000907E00501C80E116F57
:104D50000F0E126FE3EF22F00601010EC36FE0ECBD
:104D600049F0000901E012008FB615D0060173B5B5
:104D700012D00401205106011C5D040121510601DD
:104D80001D5909E21ED907E334EC47F0000903E09E
:104D90000ED9EF0E0CD08FA60DD013D90BE2060161
:104DA00073852FEC47F0000905E001D9F00E156F6F
:104DB0000F0E15D004011A5106011C5D04011B5190
:104DC00006011D590FE21AC419F51BC41AF51CC6B9
:104DD00017F51DC618F50501040E156F100E166F98
:104DE00062EF23F03FC663F640C664F647EC3AF044
:104DF0000401406F7FEC1EF0000908E03FC6FAF0A6
:104E000040C6FBF0A9EC35F0236A12003FC692F6CB
:104E100040C693F6E1EC44F08FB236D0040126513F
:104E200006011C5D0401275106011D592DE30601F1
:104E3000738329C659F42AC65AF45FC439F560C48D
:104E40003AF52BC637F52CC638F505010E0E356F31
:104E5000100E366F3DEC24F006012B5104015F5D0E
:104E600006012C51040160590FE3DCEC49F0050107
:104E70000F0E116F100E126FE3EC22F035EC0EF0F6
:104E8000C0EC0EF0080E0DD071EC41F03FC6ACF650
:104E900040C6ADF689EC1BF00401568FC0EC0EF055
:104EA000050E236E120088EC3BF0000906E00501B8
:104EB0007A0E90D8DCEC49F05CD00501D6A14CD03C
:104EC0003FC654F440C655F4C4EC35F0660E0601F6
:104ED00029250601AE6F000E06012A210601AF6FDB
:104EE000040161510601AE5D040162510601AF5932
:104EF00004E261C4AEF662C4AFF6AEC639F5AFC621
:104F00003AF529C637F52AC638F505018E0E356FF4
:104F1000170E366F3DEC24F0DCEC49F006012B5106
:104F20000601295D06012C5106012A5913E329C601
:104F300039F52AC63AF52BC637F52CC638F50501E2
:104F4000910E356F170E366F3DEC24F035EC0EF0F8
:104F5000C0EC0EF0080E0ED08FEC35F000090CE01E
:104F60000501990E37D8DCEC49F0F9EC41F0C0ECC2
:104F70000EF00F0E236E12000401568F0601010E73
:104F8000B96F77EC49F0000904E005019D0EEAEFE6
:104F900027F00401B60EF66F170EF76F26EC1DF022
:104FA000000901E1120002EC41F0C0EF0EF024C450
:104FB00019F525C41AF51CC617F51DC618F5050107
:104FC00012000401245106011C5D04012551060153
:0E4FD0001D591200116F170E126FE3EF22F041
:024FDE00C950B8
:104FE000E86E5DC570F5E3EF28F0908AC69A12006E
:104FF000DED863D9C70E5D6F68EF29F0D8D85EC5DB
:1050000062F55FC563F526D8000901E1000C55D9AA
:10501000420E62D95FC514F0156A5FC55DF5DFDF2A
:105020005EC55DF555D9010CC2D860C562F561C594
:1050300063F510D8000901E1000C3FD9D80E4CD916
:1050400061C514F0156A61C55DF5C9DF60C55DF520
:105050003FD9010C62C514F063C515F0166AD890EB
:105060001650010A01E62DD901E3000C010C64C5BC
:1050700014F065C515F0166AD8901650010A01E6BD
:1050800020D901E3000C66C514F067C515F0166A57
:105090001A6A1B6A010E1C6E64C51DF065C51EF000
:1050A0001F6A1D501A5C176E1E501B58186E1F5039
:1050B0001C58196EE8501618E8AE02D0163406D007
:1050C0001450175C155018581650195801E2000C6E
:1050D000010C7F0E05016815146E156A800ED880CC
:1050E000145614C014FD6A510D01145C02E21451EF
:1050F000120005016A511200908AC66AC79EC78CC9
:105100009D969E96C68AC950120051D805016F51CE
:105110000501666F676B6BC564F56CC565F5A7DF48
:10512000000901E1000C05016F51000839E2909A75
:105130000501030ED1D86CC514F0156A6CC55DF578
:105140004EDF6BC55DF54BDFC950E86E6FC56AF584
:105150006BC568F56CC569F5BCDF0D01136FE850D0
:1051600005016F5F0D011351146E156A145005018E
:105170006B2715506C230D011351130700080EE225
:105180000501706B20D805016DC5E9FF6EC5EAFF0A
:105190006D2B000E6E23C9CFEFFFEDD7908AC3D7DA
:1051A000010C909A0501060E97D8908A1200909AE9
:1051B000C69E0501050E90D805015D6B10DF908A33
:1051C000C9B0F5D7120070C5C9FF9EA6FED79E963E
:1051D0001200EDDF050175510501666F676B71C542
:1051E00064F572C565F543DF000901E1000C0501B6
:1051F0007551000822E2909A0501030E49D8C95062
:10520000E86E51D81351000816E20501706BDBDF20
:1052100073C5E9FF74C5EAFFEF50C95C02E0908AEC
:105220000CD00501732B000E7423712B72237507AC
:105230000D011307E7D7908ADAD7050175510008E9
:1052400026E2B5DF3AD8020E23D82DD8E850050162
:10525000755F0D011351146E156A14500501712705
:10526000155072230D011351130700080CE20501BC
:1052700073C5E9FF74C5EAFF732B000E7423EFCFEB
:105280005DF5ADDEEFD7908AC950E86ED6D7010C38
:1052900023D872C514F0156A72C55DF5A0DE71C51C
:1052A0005DF5EFEF27F075C56AF571C568F572C554
:1052B00069F50FDF0D01136F120073DF909A05017E
:1052C0001200000E145C000E1558010E1658120044
:0E52D00086DEC950908A12005D6FEFEF27F066
:0252DE0090C579
:1052E00091F50CD8146EE66E8FC591F507D8E5528E
:1052F000E7CF14F00A0DF3501424120091C59AF56B
:1053000067D8000904E0300E0501915D1200410EDE
:105310000501E76E9119E8AE02D0E73402D0E750FC
:10532000915D0DE3460EE76E9119E8AE02D091351E
:1053300003D0E750D880915502E3410E16D0610E9C
:10534000E76E9119E8AE02D0E73402D0E750915DE4
:105350000FE3660EE76E9119E8AE02D0913503D0E7
:10536000E750D880915504E3610E915D0A0F120059
:10537000000C93C591F5C2DF146EE66E92C591F5EF
:10538000BDDFE552E7CF14F0100DF35014241200E6
:1053900005019651960700090AE094C5E9FF95C5F5
:1053A000EAFF942B000E9523F6D8F2E1000C010CD5
:1053B00005019951990700090AE097C5E9FF98C5C9
:1053C000EAFF972B000E9823EBD8F2E1000C010CBA
:1053D000300E0501E76E9A19E8AE02D0E73402D02C
:1053E000E7509A5D01E2000C390EE76E9A19E8AEBB
:1053F00002D09A3503D0E750D8809A5501E2000CCC
:10540000010C9BC59AF5E4DF000901E0010C410E97
:105410000501E76E9B19E8AE02D0E73402D0E750F1
:105420009B5D0CE3460EE76E9B19E8AE02D09B3500
:1054300003D0E750D8809B5501E3010C610EE76E65
:105440009B19E8AE02D0E73402D0E7509B5D0CE335
:10545000660EE76E9B19E8AE02D09B3503D0E7508D
:10546000D8809B5501E3010C000C200E05019C5DCA
:1054700001E1010C090E9C5D01E1010C000C9DC5D0
:10548000E9FF9EC5EAFF87D801E1000C8ED883D8DA
:1054900001E1000C8AD8EFCF90F59DC5E9FF9EC5CC
:1054A000EAFFEFCF8FF51BDF9FC5E9FFA0C5EAFF3D
:1054B000EF6E010CA1C5E9FFA2C5EAFF71D801E1B9
:1054C000000C7BD86DD801E1000C77D8EFCF93F5B5
:1054D000A1C5E9FFA2C5EAFFEFCF92F54ADFA3C558
:1054E000E9FFA4C5EAFFEF6E010C0D01006B016B33
:1054F000026B036B6AD8EFCF9CF5B7DF000905E0BC
:105500000501A52B000EA623F5D75FD844D831E0BE
:105510000A0E0B6E0C6A0D6A0E6A00CD06F001CD04
:1055200007F002CD08F003CD09F08BEC49F002C082
:1055300000FD03C001FD04C002FD05C003FD45D808
:10554000EF50D00F146E156A166A176A14AE03D0A6
:1055500015681668176814500D01002715500123AF
:1055600016500223175003230501A52B000EA62376
:10557000CCD7D880FF0E0D010055FF0E0155000E4F
:105580000255000E035502E20069016900CDF3FFE8
:1055900001CDF4FF1200EFCF9AF51ADF00091200D7
:1055A000EFCF9BF52EDF00091200010E0501EA6A1C
:1055B0009D25E96E9E51EA221200010E0501EA6A5C
:1055C000A125E96EA251EA221200A5C5E9FFA6C5F0
:0455D000EAFF1200DC
:0C55D40000000000000001000700A6021B
:1055E00002000900FA0203000B00390304000C005A
:1055F000680305000D008A0306000E009F030700E4
:105600000E00B50308000F00D40309001000E803E2
:105610000A00110006040B00120022040C00130003
:1056200035040D00130047040E00140062040F003F
:1056300015007D04100016008E0411001700B80438
:1056400012001800C90413001900D904140019002D
:10565000E90415001A00010517001C001F051800B9
:105660001C002F0519001D0045051A001E005B05D2
:105670001B001F0078051C00200086051D0021006E
:105680009B051E002200B0051F002300BE05200060
:105690002400D20521002500ED0522002600070682
:1056A00023002700140624002700200625002800D8
:1056B0002D0627002A00530628002B006506290026
:1056C0002C0077062A002D0089062B002E009B0651
:1056D0002C002F00AD062D003000CA062E0032002F
:1056E000E6062F003300F706300034000E073100C5
:1056F00035001E07320036002E07330037004407FE
:10570000340038005407350039005F0736003B008D
:10571000790737003C00890738003D009D073900B4
:105720003D00A8073A003E00B2073B003F00C60715
:105730003C004000D5073D004100E4073E00420028
:10574000EE073F004300FD07400044001008410001
:1057500045001E0842004600320843004800450844
:1057600044004900570845004B006F0846004C00B4
:105770007D0847004D008F0848004E00A1084900F1
:105780004F00B3084A005100C5084B005200DB0827
:105790004C005400ED084D005500FE084E00550029
:1057A00007094F0056000F09500058002509510005
:1057B0005900360952005A00470953005C005C0941
:1057C00054005D006C0955005F00810956006000BF
:1057D000910957006200A60958006300B6096A00E3
:1057E0008200220B7A00A0005A0CB8001501441068
:1057F000C70044019111D100590125120401ED01A6
:10580000AE152D018502CC184201B102A219690121
:10581000D003821EA70116053E23DF013905B423FC
:10582000F6012006AB268B02FC08D42EAC02EE0952
:105830003E31FB02110C47363203CC0D0B3AA2036A
:10584000A0126F434C042019524ED9044B1EFF5531
:10585000E204E01F37586E051525275F7F055E2699
:10586000C9608C06DB35AA72DC06203E287B58070F
:1058700080480B850408E057799286088066319E3F
:10588000F10800738FA74109007DB1AE9C09608CBF
:1058900020B9E309C09491BE3C0A80A3CBC77A0A21
:1058A00060AE54CEBB0A80BA62D50A0B60C7A0DCDA
:1058B0006D0BE0D582E4A00BC0DFB9E9F10B20EE5F
:0858C0001DF1FFFFFFFFFFFFD8
:0858C80045D9410E34D9440E0C
:1058D00032D9430E5BD941C50CFF42C50DFF3ED105
:1058E00043C5E9F400EC1CF03DD14CD9410E23D95D
:1058F000500E3ED944C5EAF445C5EBF408EC1CF063
:1059000031D140D9490E17D9410E40D946C5F0F4DE
:1059100047C5F1F47CEC1CF00F010C6F0D6B1ED130
:1059200031D9490E08D9500E31D948C5F2F449C5CC
:10593000F3F49EEC1CF00F010C6F0D6B0FD10AD924
:10594000500EF9D8570EF7D8520E20D94AC50CFF81
:105950004BC50DFFB5EC33F04AC512FF4BC513FF25
:10596000D3EC33F00601570E0AD11BD9500E0ED9D5
:105970004CC50CFF4DC50DFFFED84CC598F64DC566
:1059800099F6E5EC48F04CC5F8F44DC5F9F443EC54
:105990001DF0F3CF0DFDF4CF0EFDD0D80DCDEAF400
:1059A0000ECDEBF408EC1CF0DDD0FBD8410EEED8A8
:1059B0004EC50CFF4FC50DFFDED84EC5FAF44FC5DE
:1059C000FBF4EBD84EC5FDF44FC5FEF4DEEC1DF044
:1059D000BBD050C5FCF4BDEC1DF09EEF2DF0E1D81E
:1059E000560EC6D851C5F8F452C5F9F443EC1DF073
:1059F0009EEF2DF0C7D8520E9ED8490EC7D805018C
:105A000053510F010C6F0D6BB5EC33F00601C4510F
:105A10000501535D0BE24CEC33F053C543F560DFF9
:105A200053C550F5D6DF53C55AF55AD8120054C5A0
:105A3000E5F455C5E6F4B9D8460EA8D854C50CFF10
:105A400055C50DFF98D854C5FAF455C5FBF4A5D833
:105A500054C5FDF455C5FEF4DEEC1DF075D056C5F9
:105A6000E7F457C5E8F4A1D8520E90D856C50CFFFC
:105A700057C50DFF80D856C5FAF457C5FBF48DD82D
:105A800056C5FDF457C5FEF4DEEC1DF05DD08DD893
:105A9000560E6ED8E7C42FF6E8C430F6E5C42DF6EE
:105AA000E6C42EF63DEC2FF0F3CF96F6F4CF97F642
:105AB000DCEF48F06ED84F0E3ED84C0E3CD8540E5A
:105AC00065D858C50CFF59C50DFFB5EC33F058C566
:105AD00014FF59C515FF00EC34F00601560E4FD0E7
:105AE0005AC5FFF423EC1EF02FD01CC65BF51DC673
:105AF0005CF57BEF2DF04DD8460E1DD8570E1BD808
:105B0000440E44D85BC50CFF5CC50DFF27D041D8BF
:105B1000520E11D8460E0FD84C0E38D81EC60CFFA8
:105B20001FC60DFF1BD0050100B9DFDF1200050104
:105B300000B9EDDF12002AD806011200F3CF4AF5B2
:105B4000F4CF4BF59FEF2CF0F3CF58F5F4CF59F588
:105B50005AEF2DF001EC23F006011200B5EC33F002
:105B600049EF33F0F3CF41F5F4CF42F564EF2CF079
:105B70000DD84CEF33F0B5EC33F04CEF33F006D8E2
:105B800049EF33F0E7DF540E9BEF2DF08C6FC3EF3E
:105B900046F0E0DF560E9BEF2DF078EC1DF09EEF07
:105BA0002DF0F0DF500E9BEF2DF0ECDF430E9BEF5E
:025BB0002DF0D6
:0E5BB200E4C5F3F3E5C5F4F3E3C5FCF30FD946
:105BC0000301F26FE8CF24F5E3C523F5330E3BD98B
:105BD000F2C3F5F34CD9E3C5F8F3E5D80301EF6F51
:105BE00001CDF7F3E3C5F6F3CBD80301F06FE8CFAF
:105BF00024F5EFC323F5340E26D9EFC3E3F5E2C550
:105C0000FCF3EDD80301F16FE8CF24F5E2C523F5ED
:105C1000350E19D9F1C3F5F32AD9E2C5F8F3C3D883
:105C20000301ED6F01CDF7F3E2C5F6F3A9D8030147
:105C3000EE6FE8CF24F5EDC323F5360E04D9EDC39E
:105C4000E2F50501060ED36F080E0301F05D0BE2CD
:105C50000501D651020B07E1D6830501010EE16F64
:105C60000501090ED36F120085EC41F00501000E0D
:105C7000E45D050EE55906E20301000EF35D0A0E30
:105C8000F45918E20501000EE45D030EE55906E241
:105C90000301000EF35D050EF4590CE20501800EC0
:105CA000E45D010EE55914E20301000EF35D020EFE
:105CB000F4590EE3D7C5E1F5D8C5E2F5D9C5E3F54A
:105CC000DAC5E4F5DBC5E5F50501050ED36F120075
:105CD0000301EE510501E25D11E2E2510301EE5DC7
:105CE0000D01006F0301F1510D01D880005502E252
:105CF000F1C300FD00510501E22712000301F0513C
:105D00000501E35D13E2E3510301F05D0D01016F55
:105D10000301F2510D01D880015502E2F2C301FDE9
:105D200001510501E327EDC3E2F51200E1050CE1A5
:105D30000501D651040B08E1D6850501E16BEDC3E1
:105D4000E2F5EFC3E3F51200B6EC41F00501D681B0
:105D50001200F5C300FD05014D0E84D801E26BD899
:105D60000501800E7FD801E266D80501000ED880BB
:105D7000E455030EE55501E25ED80D010051120015
:105D80000301F751146E156AF65162D8E8AE02D0DD
:105D9000173404D01650145C1750155803E2F6510E
:105DA000F7251200FF0C0301F951D880F85503E2E2
:105DB000F951F85D1200000C0301FA51146E156AD6
:105DC000FB5146D8E8AE02D0173404D01650145C0C
:105DD0001750155803E2FA51FB251200FF0C05017C
:105DE0004D0E40D805E30301FC39E842070B11D002
:105DF000800E38D804E30301FC390F0B0AD0000EE3
:105E0000D880E455020EE55506E30301FC39E84667
:105E10001F0BFC6F09D0050E146E0E6EFCC309F04B
:105E200097EC4BF009C0FCF30301FC5102E1010EB9
:105E3000FC6FFC511200F5C3FBF300CDFAF3BCDF9D
:105E40000D01006F12000501216F226BA8EF23F0F6
:105E5000166E176AFF0ED8801656000E175615508C
:105E600017181200D880E455010EE555120071DFB5
:0A5E70000D01016FE8CFF9F31200F5
:065E7A0006012F5130115A
:105E800003E1F36A010E3BD02DC6FDF42EC6FEF4ED
:105E9000DEEC1DF0F3CF00FDF4CF01FD0D01026B30
:105EA000036BF3CF04FDF4CF05FD02CD06FD03CD5A
:105EB00007FD2FC6FDF430C6FEF4DEEC1DF0F3CF77
:105EC00008FDF4CF09FD0D01F3500027F450012324
:105ED000000E0223032302CD03FD01CD02FD00CD00
:105EE00001FD006B166A176A0451F35C0551F45802
:105EF000065116580751175804E3F368630EF46E01
:105F0000120008CD14F009CD15F0166A176A145066
:105F1000045F1550055B1650065B1750075B04CDF8
:105F200014F005CD15F006CD16F007CD17F0D8907A
:105F3000173216321532143214500027155001232F
:105F40001650022317500323000EE96E0D0EEA6E61
:105F500004CD0BF005CD0CF006CD0DF007CD0EF005
:105F6000EECF06F0EECF07F0EECF08F0EFCF09F05E
:105F7000BAEC4AF009C0EDFF08C0EDFF07C0EDFF25
:105F800006C0EFFFFF0E0D01005D630E0159000E0C
:105F90000259000E035903E30069630E0CD0D88048
:105FA000000E0055010E0155000E0255000E03555E
:105FB00005E3006B010E016F026B036B00CDF3FF75
:105FC00001CDF4FF1200060E235C17E1020E05015D
:105FD000D35D13E30501DA510501DF5D0501DB51F6
:105FE0000501E05905E2DFC5F3FFE0C5F4FF12004B
:105FF000DAC5F3FFDBC5F4FF120029C6F3FF2AC69A
:10600000F4FF1200040163510601295D040164518B
:1060100006012A5901E2000C0401000E635D630EC3
:10602000645901E3000C010C8FB8000CF2EC1EF077
:10603000000901E1000C88EC3BF0000901E0000CD4
:1060400006011E5106011C5D06011F5106011D5966
:1060500001E2000C04012F5106011C5D04013051C6
:1060600006011D5901E2000C02EF30F00601000E9E
:10607000315D010E325906E3FF0ED8803155630EB3
:10608000325501E2000C010C040E06019E5D01E098
:10609000000CCDEC1CF0000901E1000C63C400FD14
:1060A00064C401FD0D01026B036B030E0B6E0C6AE1
:1060B0000D6A0E6A63C406F064C407F002CD08F0EE
:1060C00003CD09F08BEC49F002C000FD03C001FDD7
:1060D00004C002FD05C003FD020E0D01D89003337C
:1060E000023301330033E806F9E1060129510D01BD
:1060F000005D06012A510D01015901E2000C010C5D
:1061000033C631F634C632F6B1DF000908E033C6D3
:106110002BF634C62CF633C659F434C65AF41200A2
:1061200006016E5103E06E0701E012006C51030A94
:1061300024E0010A1EE0030A03E0010A3CE0120029
:106140006E6B6B5106E0130E6B5D03E0150E6B5D1D
:1061500002E16F6B10D021D906016B510F010C6F5A
:106160000D6BB5EC33F049EC33F006010A0E6F6F9E
:106170000AD080D80601030E10D01ED806016F5138
:1061800004E06F0702E0020E08D06B2B6A51D88042
:106190006B5505E3190E6E6F010E6C6F12006DC624
:1061A000B9F677EC49F00601060E6E6FF6D849ECA9
:1061B00033F006016C6B12000601060E6E6F6B5118
:1061C000180A54E00F0A50E0010A4CE0020A48E0C5
:1061D000060A44E0030A40E0010A3CE01F0A38E0F6
:1061E000010A34E0030A30E0010A2CE0070A28E043
:1061F000010A24E0030A20E0010A1CE00F0A18E06B
:10620000010A14E0030A10E0010A0CE0070A08E0A2
:10621000010A04E0030A2CE18C9012008C96120013
:106220008C9A12008C9C12008C9E12008C9812008A
:106230008C9412008C9212008D9E12008D9C120084
:106240008D9A12008D9812008D9612008D94120076
:106250008D9212008D9012008F9012008F94120078
:106260008F9212008F9612008F981200909E12004B
:106270006E6B12000601060E6E6F6B51180A54E029
:106280000F0A50E0010A4CE0020A48E0060A44E026
:10629000030A40E0010A3CE01F0A38E0010A34E04A
:1062A000030A30E0010A2CE0070A28E0010A24E092
:1062B000030A20E0010A1CE00F0A18E0010A14E0BA
:1062C000030A10E0010A0CE0070A08E0010A04E0F2
:1062D000030A2CE18C8012008C8612008C8A12003A
:1062E0008C8C12008C8E12008C8812008C84120010
:1062F0008C8212008D8E12008D8C12008D8A1200FD
:106300008D8812008D8612008D8412008D821200FD
:106310008D8012008F8012008F8412008F821200F5
:106320008F8612008F881200908E12006E6B120002
:1063300006016951180801E21200695101E16A6B16
:1063400069516A5D02E269C66AF66A51180802E29A
:10635000180E6A6F6C511BE1A1EC35F0000901E0E9
:1063600012000401F66BF76B26EC1DF0000901E04A
:1063700012000601695101E112008F50020B01E089
:10638000010E6D6F69C66BF66E6B010E04D06A6B01
:106390006F6B6E6B030E6C6F12000601570E8C6FE5
:0E63A000C3EC46F006014B0E8C6FC3EF46F0C7
:0263AE00A7C581
:1063B00065F657EC3AF0F3CFAEF5F4CFAFF568D809
:1063C000F3CF14F0F4CF15F0010E1426000E1522B1
:1063D00014C0F3FF15C0F4FF1200A8C577F6A9C5D5
:1063E00078F69FEC48F0F3CFA8F5F4CFA9F517D9CC
:1063F0000D01006FE8CFA7F5D7EF31F00501AA51E5
:10640000AB1116E0AC51AD1113E0AAC563F6ABC5F4
:1064100064F647EC3AF0146EE66EACC563F6ADC5B3
:1064200064F647EC3AF0E552E7CF14F0145C03E071
:10643000F368F4681200AAC5AEF5ABC5AFF528D86D
:10644000F3CF00FDF4CF01FDACC5AEF5ADC5AFF5A2
:106450001FD8F3CF02FDF4CF03FD0D01F450011955
:10646000E8AE02D0013504D00051025D015103595C
:1064700006E20251005D146E0151035505D0005132
:10648000025D146E0351015514C0F3FFF46E120047
:10649000AEC563F6AFC564F647EC3AF00501B26FDE
:1064A000AEC5B0F5AFC5B1F556EF32F0B0C577F671
:1064B000B1C578F69FEC48F0F3CFB0F5F4CFB1F565
:1064C0000501B25100080AE2B2050601656F57ECFA
:1064D0003AF0F3500501B05FF450B15BB007000E25
:1064E000B15BB2C5B3F517D8F3CF14F0F4CF15F004
:1064F000B0C508F0B1C509F0F3CF0DF0F4CF0EF040
:106500003AEC4BF008C00CFD09C00DFD08C0F3FFCC
:1065100009C0F4FF12000501B3510A0A08E0030A9A
:1065200004E0090A06E10A0E05D0640E03D0C80E85
:1065300001D0140EF36EF46A1200B4C577F6B5C537
:1065400078F69FEC48F06BD80501B36F8BEF32F013
:106550000D010E6B0F6B0501B651000809E2B6057F
:106560000601656F57EC3AF0F3CF0EFDF4CF0FFD47
:10657000B6C5B3F5D0DFF3CF16F0F4CF17F0B7C53B
:1065800008F0B8C509F0F3CF0DF0F4CF0EF046ECEB
:1065900044F006C014F007C015F0010E1426000EDA
:1065A000152214500D010E2715500F230ECDF3FFA9
:1065B0000FCDF4FF12003FC6ACF540C6ADF5B9C52E
:1065C000AAF5BAC5ABF51ADFF3CF04FDF4CF05FD8C
:1065D0000D01F43404E204510208000E055504E3F1
:1065E000041D03E1051D01E1010C000C01EC23F089
:1065F0000601420E8C6FC3EC46F00601490E8C6F0B
:10660000C3EC46F006014E0E8C6FC3EC46F0BBC5E2
:106610000CFFBCC50DFFB5EC33F049EF33F0F3CF01
:0A66200063F6F4CF64F647EF3AF09A
:06662A000D01006B070EDC
:10663000016F0F0105510527640E055D04E3640E2B
:10664000055F0D01002B0D01005100270107F1E14D
:10665000005112000D01010E296F640E2A6F0F0107
:1066600006510CE006AF03D00D012A5129270F0176
:10667000065106270D012A912A43F1D70D01295110
:10668000FE0BE84212000F010751036F046B96EFF7
:1066900033F006013B0EE8D00601200EE5D00601DE
:1066A0000D0E8C6FC3EC46F006010A0EDDD00F0113
:1066B00008390F0B0F01096F04D808CF09FF61EFEC
:1066C00033F00F0E0F0109170951090802E2370EC6
:1066D00001D0300E09250601C7D0300E0F010A1176
:1066E0000601C2D00D01300E416F0F010151035D53
:1066F000025104590AE30151035F0251045B0D0189
:10670000412B0F01010E006FF0D7005104E041CD85
:106710008CF6C3EC46F012000F01010E006F37EF4C
:1067200034F00A0E0F01A3D88CEF33F00F01010EE5
:10673000006F91EF33F0640E0F0199D891EF33F0B1
:106740000F01E80E016F030E026FCCDF9BEF33F0F9
:106750000F01100E016F270E026FC4DFA0EF33F0A0
:106760009BDF0BCF08FF57EF33F096DF0CCF0EFF08
:106770000DCF0FFFBCEF33F00ECF03FF0FCF04FFA1
:106780000F01006BA8EF33F011CF03FF0F01046B73
:1067900063D80F0110510F01066F5CDF0F01036F0B
:1067A000046B96EF33F012CF03FF13CF04FF050EF7
:1067B0000F0B0F0102E05FD8FEE10F01006B6CDFF1
:1067C000BFDF06012E0E8C6FC3EC46F012CF03FF25
:1067D0001F0E0F010317046B640E0403F3CF04FFB5
:1067E0000303F3CF03FFF4500427100E0327000E1A
:1067F0000423050E0F0B02E03ED8FEE196EF33F0C6
:1068000014CF03FF15CF04FFC80E0D6E0E6A14CF10
:1068100008F015CF09F03AEC4BF008C003FF09C0AF
:1068200004FFC80E086E096A03CF0DF004CF0EF006
:1068300046EC44F006500F01145F0750155B0CD86E
:1068400014CF03FF15CF04FF010E0F0B0F0102E061
:1068500012D8FEE196EF33F0006B1EDF6CDF06010D
:106860002E0E8C6FC3EF46F08C6FC3EF46F0016FB6
:10687000026B72EF33F0D89004330333E806120052
:10688000120000C663F601C664F647EC3AF00D014B
:10689000006F00C6AEF501C6AFF548EC32F0F3CF9D
:1068A00001FDF4CF02FDF3CF56F6F4CF57F600CD3D
:1068B00055F61FEC40F0F3CF03FDF4CF04FD01ECDF
:1068C00023F00601440EF3D8FAD800CD67F695EC14
:1068D0003AF001CDBBF502CDBCF5F6EC32F001CDBE
:1068E00005F602CD06F600CD04F671D803CD07F605
:1068F00004CD08F69ED803CD5BF604CD5CF658ECCB
:1069000040F00D01056B060E055D1DE24FEC33F006
:106910000501060E6F6F0501060E6D6F0D0E6E6F91
:1069200003CD6BF504CD6CF585EC28F00601060E61
:10693000026F0D0E036F08D8060E0D010327000E1F
:106940000423052BE0D71200C1D8FF080EE1060191
:10695000550EADD84E0EABD8550EA9D8530EA7D8AC
:10696000450EA5D8440E63EF35F0B0D8030B0601F1
:10697000A86F2BEC48F0AAD8800B01E0010E0601AD
:10698000B86F51EC49F0A2D8800B16E09FD8400BAD
:1069900001E0010E0601B06F1CEC49F08BD8010E2E
:1069A000EB500601B66F01EC4BF084D8020EEB50B1
:1069B0000601B46FE6EC45F07DD8030EE926000E23
:1069C000EA22EECF98F6EDCF99F6E5EF48F005C64E
:1069D000B7F506C6B8F504C6B6F5A8EC32F0F3CFA5
:1069E0000CFDF4CF0DFD0601460E61D8520E6BD89A
:1069F0000CCD0CFF0DCD0DFFB5EC33F006012D0EC7
:106A000062D804C6B3F58BEC32F0F3CF14F0F4CFB8
:106A100015F01406000E155A14500D010C271550D0
:106A20000D230CCD0EFF0DCD0FFFBCEC33F049EF65
:106A300033F00601410E3BD8440E39D8440E37D806
:106A4000520E41D807C60CFF08C60DFFB5EC33F057
:106A500049EF33F0050100510AE05CEC48F086ECA8
:106A600049F047EC49F01BEC4BF027EC46F01200E4
:106A7000050100511BE001EC23F00601530E17D86D
:106A8000460E15D81CD809C679F60AC67AF6C4ECA3
:106A900048F009C663F60AC664F647EC3AF0060108
:106AA000676F95EC3AF0FCEC48F0D4DF12000BD89D
:106AB0000601120002C6E9FF03C6EAFF12004D0EEE
:106AC00002D84CEF33F08C6FC3EF46F0F3DFEF509A
:026AD0001200B2
:0E6AD20085EC3AF0000921E0040103510601B1
:106AE000615D1CE061C680F486EC0DF0F3CFFEF52D
:106AF000F4CFFFF50501F350F41001E0FC87FEC56B
:106B000019F5FFC51AF5060161510501176F186BDC
:106B1000A10E0501156F166B62EC23F01200050142
:106B2000FC51040B03E106018D510AE006018D6B57
:106B30000501040E116F290E126FE3EC22F0010C17
:106B4000000C235004E0010A02E00E0A01E1000CEF
:106B5000010C0001FA51FB1116E03FC619F540C6C1
:106B60001AF5FAC017F5FBC018F505013C0E156FB4
:106B7000280E166F62EC23F0FAC0FEF5FBC0FFF59D
:106B80000501FC87FC8B120054C4F8F055C4F9F0E1
:106B900004015651030B0001F76FE8500501196F0E
:106BA0001A6B54C417F555C418F50501A00E156FDE
:106BB000280E166F62EF23F0410E0401085D01E01C
:106BC000000C060129510401615D06012A510401EE
:106BD000625901E3000C88EC3BF0000901E0000C75
:106BE0000601C2A1000CC2BD000CCDEC1CF00009D6
:106BF00001E1000C1CEC48F00001F75D12E1F8C067
:106C0000B9F5F9C0BAF5DBEC32F000090AE106018A
:106C100029510601AE5D06012A510601AF5901E373
:106C2000000CC9EC44F0010C1CEC48F00001FC5DC8
:106C300001E1000C0601DD0E42D801E0010C040167
:106C4000E20E44D801E0010CFCC0A9F645EF48F083
:106C5000FDC06DF3FEC06EF391EC11F0000901E090
:106C6000000C0601830E2BD801E0010C0401E70E95
:106C70002DD801E0010CFDC08DF4FEC08EF496EC21
:106C80000EF0000914E0060173B310D0FDC0E9FF57
:106C9000FEC0EAFF030EE926000EEA22EECF33F62D
:106CA000EDCF34F680EC30F0FCEC48F0010C05013F
:106CB000920E116F270E126FE3EC22F0000CBC6FE6
:106CC000270EBD6F1FEC43F000091200EE6F270E78
:0A6CD000EF6F5EEC1CF000091200EB
:066CDA00060126512711FE
:106CE00003E1F36AF46A120026C600FD27C601FD1F
:106CF0000D01026B036BF30E0B6E0C6A0D6A0E6ACC
:106D000026C606F027C607F002CD08F003CD09F02D
:106D10008BEC49F00D01036B03C0F3FF04C0F4FFDB
:106D200012009E9C300EC16EBA0EC06E98EF36F007
:106D3000020E0D01006F016B040E026F0601286B3D
:106D40005CD8C3500D010027C45001230207025133
:106D50000008F4E300CD24F601CD25F6020E0F0B5A
:106D6000060105E0D89025332433E806FBE1120044
:106D7000060173AB13D0739B20C626F621C627F6F7
:106D8000ACDFF3CF20F6F4CF21F622C626F623C6D9
:106D900027F6A3DFF3CF22F6F4CF23F646D8060179
:106DA0001C51205D1D51215927E21CC620F61DC62D
:106DB00021F61EC622F61FC623F60401265106013F
:106DC000205D040127510601215916E322C62FF642
:106DD00023C630F620C62DF621C62EF63DEC2FF048
:106DE000F3CF29F6F4CF2AF68FB206D029C633F6B0
:106DF0002AC634F680EC30F01200C26A060128512F
:106E00001F0BF36EF346F346830EC214F310C26EEB
:106E1000C280C282C2B2FED7E00ED880C3540F0E29
:106E2000C45402E2C36AC46A12000D01040E006F6A
:106E3000020E016F026B036F046B0601140E286FC4
:106E4000DCDFC3500D010127C45002230601245189
:106E5000C35C2551C45807E324510D01015F0601AD
:106E600025510D01025B0601160E286FC6DFC350C7
:106E70000D010327C450042306012451C35C25518E
:106E8000C45807E324510D01035F060125510D018C
:106E9000045B0D01000700510008CFE301CD1CF693
:106EA00002CD1DF6020E0F0B060105E0D8901D3332
:106EB0001C33E806FBE103CD1EF604CD1FF6020EDF
:106EC0000F0B060105E0D8901F331E33E806FBE1E7
:026ED0001200AE
:0E6ED2000501000EDA5D050EDB591DE2E2C57A
:106EE00087F6BFD80601836FE3C587F6BAD80601D7
:106EF000846FE8CF24F583C623F51F0E0501216FAB
:106F0000226BA8EC23F00601866B856B0501E26B12
:106F1000E36B0501040E09D00501E10505E1AFD8D9
:106F2000E16B0501010E01D0BFD8D36F120085ECD3
:106F300041F00501330ED880DA55010EDB5507E22A
:106F40000501330ED880DF55010EE05503E3ACD8C0
:106F5000D36F1200070E0601855D2AE0852B85514F
:106F6000070802E2070E856F100E8503F3CFE2F5E6
:106F7000FF0E835D14E10501E251146E156AE251C2
:106F800089D8E8AE02D0173404D01650145C1750DC
:106F9000155803E2E251E2271200E2691200835120
:106FA0000501070B5DE0E243E29FE806FCE1120009
:106FB000856B0501E26B070E0601865D25E0862BD9
:106FC000100E8603F3CFE3F5FF0E845D14E1050197
:106FD000E351146E156AE3515DD8E8AE02D0173460
:106FE00004D01650145C1750155803E2E351E32700
:106FF0001200E369120084510501070B31E0E343FD
:10700000E39FE806FCE112000501E10527E137D81E
:107010000501660ED880DA55010EDB550CE304013C
:107020000351050808E3080E0501D95D04E3080EC5
:107030000501E35D05E20501E16B0501010E0CD0E0
:10704000D7C5E1F5D8C5E2F5D9C5E3F5DAC5E4F56C
:10705000DBC5E5F50501050ED36F120025D8D36F0A
:107060001200C00E0601871501E0FF0C87BB000C63
:1070700087B9010C87B7020C87B5030C040CD7C580
:10708000DCF5D8C5DDF5D9C5DEF5DAC5DFF5DBC53C
:10709000E0F51200166E176AFF0ED8801656000E25
:1070A0001756155017181200B6EC41F00501050EE1
:0270B0001200CC
:0E70B2000501DA69630EDB6FC9D80301FD6FBB
:1070C000080ED9D802E0DBD8FEE10501D96F050131
:1070D000E36F800ED0D802E0D2D8FEE10301FE6F4C
:1070E000010EFF6F100EC7D802E0C9D8FEE10501FE
:1070F000D86F0501E26F0501020ED36F120085EC17
:1071000041F00501660ED880E455010EE55518E3FF
:10711000D7C5E1F5D8C5E2F5D9C5E3F5DAC5E4F59B
:10712000DBC5E5F50501030ED36F0501330ED880ED
:10713000E455010EE5556EE30501050ED36F12000F
:107140000F0E0301FF5D10E2FF2B0501E6510AE07F
:107150000301FF2B0501FF0EE45D630EE55902E319
:107160000301FF2B0BEF39F0010EFF6F54D8030121
:10717000FE510501E35D47E2E3C500FD0501E6516F
:1071800013E00D01010E006F020E0401035D02E227
:107190000D01002B0501FF0EE45D630EE55925E3AB
:1071A0000D010051002721D0400E0D01005D07E3C5
:1071B00004016751010B03E00D01200E15D0200ED4
:1071C0000D01005D07E304016751010B03E00D01B0
:1071D000100E0AD0100E0D01005D07E30401675187
:1071E000010B03E00D01080E006F0501E3510301DF
:1071F000FE5D0D01005D04E200510501E327120070
:10720000FEC3E3F51200D8C5E2F5D9C5E3F50501E3
:10721000030ED36F1200100E0301FF5D0AE2100E81
:10722000FF03F35028D802E02AD8FEE10501E26FFF
:107230001200FF0E20D802E022D8FEE10501E26F25
:107240000301FD51000802E20501E22B12000401D6
:107250000351050A0EE0030A0CE0050A09E0070ADB
:1072600007E0040A04E0010A02E0030A03E1000C5B
:10727000010C020C030CFDC3E7FFE7521200E842C9
:067280007F0BE70612007F
:0A728600D8D8500EC9D8530EC7D84F
:10729000490ECED8010BC6D0D3D8410EC9D8400B69
:1072A00001E0010EBFD0CCD84D0EC2D8800B01E05A
:1072B000010EB8D0C1D84D0EB2D8440EC7D808C4FC
:1072C0008CF6C3EC46F049EF33F00501020EF56F82
:1072D0000501000EF36F0D0EF46F0501F16BF26BFB
:1072E0001FEC3FF0A9D8530E9AD84E0EAFD800CD60
:1072F0000CFF01CD0DFFB5EC33F049EF33F09CD816
:10730000530E8DD84C0E94D8200B01E0010E8AD07C
:107310000601C1515A0A4EE0020A47E00F0A40E056
:10732000030A39E0060A32E01E0A2BE00A0A24E0CA
:10733000030A1DE0010A16E0070A0FE0010A08E04F
:10734000030A01E0120022C400FD23C401FD37D06E
:107350002AC400FD2BC401FD32D01EC400FD1FC491
:1073600001FD2DD024C400FD25C401FD28D020C47A
:1073700000FD21C401FD23D01AC400FD1BC401FD82
:107380001ED026C400FD27C401FD19D028C400FD6D
:1073900029C401FD14D01CC400FD1DC401FD0FD083
:1073A0002CC400FD2DC401FD0AD018C400FD19C471
:1073B00001FD05D004012E510D01006F016B3CD879
:1073C000540E2DD8560E42D8C1C68CF6C3EC46F0EA
:1073D00000CD0EFF01CD0FFFBCEC33F049EF33F0D1
:1073E0002BD8410E1CD84B0E1AD8490E18D8500E67
:1073F0002DD814C40CFF15C40DFFB5EC33F00601F5
:10740000570E24D84CEC33F016C45BF517C45CF56A
:107410007BEF2DF00501005101E04CDF120016D882
:10742000060112000F010A6F6DEC33F049EF33F0E3
:107430000DD804010951120001EC23F006011200DD
:10744000FBDF4D0EECDF540E0FEF3AF08C6FC3EF05
:0274500046F004
:0E74520006016251030A17E0070A15E0010A5D
:1074600013E0030A11E0010A0FE00F0A0DE0010A20
:107470000BE0030A09E0080A06E0030A03E0010A38
:1074800005E1020C000C010C625112000F0C0D0101
:107490000C6B0C51ACD806016351145C6451155847
:1074A00003E20D010C2BF5D70D010C511200060162
:1074B00065519DD814C0F3FF15C0F4FF1200600E93
:1074C000166E970E176E000E186E66C619F01A6AC1
:1074D0001B6AD89019361A361B3616501924F36ECB
:1074E00017501A20F46E18501B20F86EF4CFF7FFD7
:1074F000F3CFF6FF0900F5CF14F00800F5CF15F033
:1075000014C0F3FF15C0F4FF120006015F51615D66
:1075100001E1000C040E605D01E2000C0B0E5F5DEA
:1075200001E3000C5FC661F6010C01EC23F00601DB
:10753000420E8C6FC3EC46F006014E0E8C6FC3EC0E
:1075400046F067C607FF43EC33F049EF33F022D82B
:107550000601685D10E05F510501196F1A6B0601A5
:1075600068510501176F186BCE0E0501156F166B6C
:1075700062EC23F0000C5FC661F6010C0D01016B9B
:1075800080BA018780B4018580B6018381B0018112
:1075900001511200F3DF0601626F5BDF0D01006F26
:1075A000E85006015F5D07E10401F66BF76B26EC1E
:1075B0001DF0000905E000CD5FF60601606B0DD0FF
:1075C00006016051146E156AD890155004E6FF0E3E
:1075D000145C000E155801E2602B0D0100511200E1
:1075E0000501005103E003C467F69FDF1200E96E56
:1075F000EA6AD890E936EA36BD0EE926050EEA2297
:0A760000EECF14F0EFCF15F01200EA
:06760A009FC6A0F69ED809
:10761000000901E11200020E0501EC6FED6BF0ECC8
:107620003EF00D01006F06019F511EE10501100E95
:107630006F6F0501010E6D6F0D0E6E6F0D01005124
:10764000100DF3CF6BF5F4CF6CF585EC28F00D0140
:1076500001510AE1051D01E1061D06E0A7D8052B31
:10766000000E0623B4EF3BF090D89FC601FD9ED8D4
:1076700006019F5105E1010E0D01056F066B14D047
:107680003FC605FD40C606FD1CC607FD1DC608FD1C
:107690001EC609FD1FC60AFD29C60BFD2AC60CFD24
:1076A0002BC60DFD2CC60EFD5FD806019F51010AA9
:1076B0001FE16BD80D01810E016F78D8D4C505FD8F
:1076C000D5C506FD1CEC48F00D01076F8F50020B6D
:1076D00001E0010E086FFFEC4AF00D010A6FD2ECD9
:1076E00045F00D010B6F17EC49F00D01096F3CD807
:1076F00000CDF0F5020E0501EE6FEF6B02EF3FF0EB
:10770000040E06019E5D03E10601A06B1FD8120066
:1077100006019E5102E0040A01E1000C010C01EC9B
:1077200023F00601460E8C6FC3EC46F006014C0EAA
:107730008C6FC3EC46F00601540E8C6FC3EC46F020
:107740009EC60AFF6DEC33F049EF33F006019E51FF
:10775000A05D01E1000CA0C69EF601D8010C050158
:10776000005101E0DCDF12000501100E756F05010C
:10777000010E736F0D0E746F0D010051100DF3CFDC
:1077800071F5F4CF72F5E9EF28F00D01002B100E22
:10779000E66EE66AE66A010EE66E0D0EE66E20EC17
:1077A0004BF0146E050EE15E1450120074C602FD1B
:0A77B00075C603FD76C604FD120045
:0677BA00DACFE4FFE2CF8C
:1077C000DAFFE9CFE4FFEACFE4FFF6CFE4FFF7CF3B
:1077D000E4FFF8CFE4FFF3CFE4FFF4CFE4FFFACF08
:1077E000E4FFFBCFE4FF00EE00F0140EE80403E337
:1077F000EECFE4FFFBD7E652CD90CECF3DF6CFCF14
:107800003EF6C60E06013D27E00E3E233EC6CFFFE4
:107810003DC6CEFFCD809E90D6CF3DF6D7CF3EF66B
:10782000D76AD66A3DC638F63EC639F6060170B745
:107830005DD00601BB0E385D000E395955E30401D9
:107840001A5106011C5D04011B5106011D594CE330
:1078500004011A510601365D04011B510601375916
:1078600043E306011C5106011E5D06011D51060180
:107870001F593AE2060138513A5D39513B5906E346
:1078800038513A5D3D6F39513B5905D03A51385D19
:107890003D6F3B5139593E6F010ED8803D55000E6A
:1078A0003E551CE33C2B3C51246E256AD890255054
:1078B00004E6060E245C000E255811E3060E3C6F0C
:1078C000080E086E096A38C60DF039C60EF046EC8F
:1078D00044F006C03FF607C040F601D03C6B38C606
:1078E0003AF639C63BF602D006013C6B06017097AA
:1078F0001CC636F61DC637F670810601352B35518C
:10790000246E256AFA0E245C000E25580BE3356BB5
:107910000601707570B506D070830601742B000ED9
:1079200075237623E55200EE13F0140EE80403E30A
:10793000E5CFEDFFFBD7E5CFFBFFE5CFFAFFE5CFC6
:10794000F4FFE5CFF3FFE5CFF8FFE5CFF7FFE5CF95
:10795000F6FFE5CFEAFFE5CFE9FFE5CFDAFF11005B
:10796000236A0501FC6B1200235027E00501FB513F
:10797000000802E2FB07120015EC37F00401265163
:1079800006011C5D0401275106011D5916E31EC6A0
:107990002FF61FC630F61CC62DF61DC62EF63DEC82
:1079A0002FF0F3CF29F6F4CF2AF68FB206D029C6EE
:1079B00033F62AC634F680EC30F005010A0EFB6F70
:1079C0002350010A06E0030A04E0060A02E0010A65
:1079D00006E18FEC35F0000902E00F0E236E235014
:1079E00006E0040A04E00B0A02E022EC23F0235034
:1079F0000F0A2AE0070A25E00E0A19E0030A14E03C
:107A0000010A0FE0060A0AE0030A05E0010A1EE186
:107A100042EC1AF01BD0A8EC40F018D07EEC40F0FD
:107A200015D081EC26F012D061EC26F00FD053EC8B
:107A300027F0020E0501D35D09E10501090EFB6F78
:107A400005D0F9EC49F002D024EC3EF00F0E235C97
:107A500003E10501190EFB6F12000D01206B0001FF
:107A6000010EFC6F14EC36F0000903E00D01010E6D
:107A7000206F0001060EFD6F030EFE6F28EC36F03E
:107A8000000903E00D01010E206F2FEC47F0000903
:107A900003E00D01010E206F0D01205104E1FCEC0B
:107AA00042F00D01206F205106E190EC10F08DECBA
:107AB00020F00501FC6B0D012051120051DF060181
:107AC0003F6B406B0601816B826B550E0401085DB4
:107AD00005E10401410E4A6FCDEC1FF03FEC0EF0C2
:067AE00003C461F6120070
:0A7AE6000601000ED8807D55400E09
:107AF0007E5544E20401F66BF76B26EC1DF000099D
:107B00003FE17DC681F67EC682F60601000E815FEA
:107B1000400E825B030ED89081378237E806FBE186
:107B200068EC4AF081C663F682C664F647EC3AF028
:107B30000D01026FE8CF68F6A7EC3AF0000920E0EB
:107B400081C63FF682C640F651EC20F0000906E0FF
:107B50003FC6A1F640C6A2F690EF42F00601615181
:107B60000501196F1A6B0D0102510501176F186B92
:107B70006C0E0501156F166B62EF23F06DEC4AF089
:107B800012000D01800E006F016B81A602D0005122
:107B9000011356D80D01009100430051F6E1015147
:107BA00012000D01800E006F9396060180510D01A9
:107BB000001502E08A8601D08A9642D80D01009114
:107BC00000430051F2E18A869386120081C6ACF52B
:107BD00082C6ADF53FC6AAF540C6ABF5FEEC31F066
:107BE000F3CF04FDF4CF05FD0D01800EF4140CE17C
:107BF000053504E204510208000E055505E381C66F
:107C0000F3FF82C6F4FF12003FC6F3FF40C6F4FF45
:107C1000120081B61200F29E2CEC46F081A6FED72F
:107C20000FD82CEC46F0ADDF06017E6FAADF06010F
:107C30007D6FA7DF06017F6F06017087F28E12004D
:087C40002CEC46F02CEF46F09D
:087C4800DCEC49F0000903E047
:107C500005013C0E9CD052EC47F0000901E01200F7
:107C60002FEC47F0000901E012000501FCAD0DD03A
:107C7000FC9D0601460E8C6FC3EC46F00601540EC7
:107C80008C6FC3EC46F049EC33F014EC30F0000993
:107C900023E063C439F564C43AF529C637F52AC62A
:107CA00038F50501460E356F230E366F3DEC24F096
:107CB0002FC419F530C41AF51CC617F51DC618F5E2
:107CC0000501470E156F230E166F62EC23F00601B7
:107CD000040EA06FA6EC3BF006019E5114E00601D5
:107CE0004B0EBC6F230EBD6F1FEC43F0000901E08B
:107CF00012000401640EEE6F230EEF6F5EEC1CF0B9
:107D0000000901E01200420E0401085D04E00401D4
:107D10005651800B0CE10001060EFD6F030EFE6F45
:107D200028EC36F0000903E00501780E28D00501A3
:107D3000FCAF12D0FC9F29C62DF52AC62EF53FC6F2
:107D40002BF540C62CF50501F00E296F230E2A6F86
:107D5000F1EC23F02AEC35F00501FC51100B03E1A6
:107D6000FC51020B03E00501050EE66F060173B737
:107D700007D0FCEC42F0000903E00501F50E07D046
:107D80000501FC6B060173937395236A1200116F52
:087D9000230E126FE3EF22F055
:087D98007F94A698A998608869
:107DA00012000501000EE75D040EE85901E3000C26
:107DB000010C0501000EE95D040EEA5901E3000C17
:107DC000E9C514F0EAC515F0000ED8801456040E6B
:107DD0001556EB51145C000E155801E3010C000C14
:107DE0000DD8EDC514F0156A1450636EECC562FF32
:107DF0007F6A7F800000615000D012007FB2FED702
:107E00007F941200FBDFEEC5E7F5EFC5E8F5C9DFAB
:107E1000000901E1000CEFC514F01450636EEEC5CB
:107E200062FFF0C561FF7F6A7F84F29E550E7E6E11
:107E3000AA0E7E6E7F8206017087F28E010CF5C558
:107E4000EBF5F1C5E9F5F2C5EAF5B3DF000901E1AB
:107E5000000C0501F551F507000815E2F1C5ECF538
:107E6000F2C5EDF5F12B000EF223BADFE66E050147
:107E7000F3C5E9FFF4C5EAFFF32B000EF423E55246
:107E8000E750EF6EE6D7010CFAC5EBF5F6C5E9F55C
:107E9000F7C5EAF58EDF000901E1000C0501FA5192
:107EA000FA0700081DE2F8C5E9FFF9C5EAFFF82B5B
:107EB000000EF923EFCF29FDF6C5ECF5F7C5EDF57A
:107EC0008FDF0D01295D07E029CDF0F5F6C5EEF550
:107ED000F7C5EFF597DF0501F62B000EF723DED788
:027EE000010C93
:0E7EE20006018D6B0601716B726B81A403D0DB
:107EF000010E716F726B120085AA010C85AC010C2A
:107F000082EF3FF087A0010C000C38D81FD84ED864
:107F100006017151721101E101D8120081A40CD047
:107F200006018E515BD801E65ED80FE28E518E2B92
:107F300019080BE18D8B1200020E06018E5D04E321
:107F4000190E8E5D01E28D898E6B120085BA0CD000
:107F500006018F5143D801E646D80FE28F518F2B8F
:107F600019080BE18D871200020E06018F5D04E3F4
:107F7000190E8F5D01E28D858F6B120087B00CD0DA
:107F8000060190512BD801E62ED80FE29051902B8C
:107F900019080BE18D831200020E0601905D04E3C7
:107FA000190E905D01E28D81906B120085BC0CD0A2
:107FB0000601915113D801E616D80FE29151912B89
:107FC00019080BE18D8B1200020E0601915D04E38E
:107FD000190E915D01E28D89916B1200146E156A84
:107FE000D89015501200FF0E145C000E15581200A8
:107FF0000D01006B100E016F000E005D400E015967
:108000000CE200CD5EF501CD5FF5FEEC27F0800EB1
:108010000D010027000E0123EFD70501606B400E14
:10802000616F14EC28F00501606B800E616F14EC39
:1080300028F00501606BC00E616F14EF28F056C682
:1080400016F057C617F050D84FD84A0E186E970E34
:10805000196E000E1A6E55C61BF01C6A1D6AD89068
:108060001B361C361D3618501B24F36E19501C206D
:10807000F46E1A501D20F86EF4CFF7FFF3CFF6FF21
:108080000900F5501624146E0900F550172014C08D
:10809000F3FFF46E120059C656F65AC657F658C684
:1080A00055F6CDDFF3CF5BF6F4CF5CF658EF40F03A
:1080B0000501240E6F6F05010C0E6D6F030E6E6FC0
:1080C0005BC66BF55CC66CF585EF28F00501240EE8
:1080D000756F05010C0E736F030E746F5DC671F53D
:1080E0005EC672F5E9EF28F0060E1702F3CF17F01F
:0C80F0001602F3CF16F0F4501726120011
:0480FC000F0E236ED2
:108100000401E40EF66F070EF76F26EC1DF0000970
:1081100001E11200DCEC35F0000901E1120061C45C
:1081200039F562C43AF529C637F52AC638F505018E
:10813000F80E356F070E366F3DEC24F00601739391
:1081400073950501FC89FC83FC8F040E236E1200DD
:1081500052EC47F0000901E012000601100EBC6F5E
:10816000040EBD6F1FEC43F0000901E01200040192
:10817000150EEE6F040EEF6F5EEC1CF0000903E0CD
:108180000F0E236E120004015651030B0001FC6F09
:1081900014EC36F0000901E012000D01560E116FCB
:1081A000040E126F420E0401085D04E004015651F2
:1081B000800B05E10D01060E116F030E126F11CD3C
:1081C000FDF012CDFEF028EC36F0000901E01200BF
:1081D0000601C2B102D00F0E13D00501FCA909D0CF
:1081E0000501420E116F040E126FE3EC22F0040E33
:1081F00007D0CDEC1CF0000902E0020E01D00F0EFA
:04820000236E1200D7
:0C8204000501D42B000ED523D8EC41F06E
:108210002DEC4AF00501000E73D802E3D68124D07C
:10822000D351060A1FE00F0A1DE00C0A18E0010AEC
:1082300013E0070A0EE0010A09E0030A04E0010A5C
:1082400013E126D811D059EC38F00ED07FEC38F07D
:108250000BD069EC37F008D097EC37F005D0D9ECAB
:108260002DF002D034EC2EF0FCEC41F00501D6A14B
:108270000ED085EC41F00501000ED880E455030EC8
:10828000E55505E20601010E9F6F05EC3BF012007B
:108290000501DF69630EE06F660E32D81EE3E1C5AB
:1082A000D7F5E2C5D8F5E3C5D9F5E4C5DAF5E5C5F6
:1082B000DBF5E1050AE1D7C5DCF5D8C5DDF5D9C5A3
:1082C000DEF5DAC5DFF5DBC5E0F5030ED36F330E5F
:1082D00017D806E3050ED36F1200010EE16FD36FBE
:1082E00012000501D36BD46BD56BD66BDF69630EBF
:1082F000E06FDFC5DAF5DB6FDFC5E4F5E56F12008F
:0A830000D880E455010EE555120087
:06830A000501DA51050136
:10831000E45D0501DB510501E55924E2E1C5D7F52E
:10832000E2C5D8F5E3C5D9F5E4C5DAF5E5C5DBF571
:10833000E10513E10501DF510501E45D0501E051AF
:108340000501E5590AE2D7C5DCF5D8C5DDF5D9C583
:10835000DEF5DAC5DFF5DBC5E0F50601530EBF6FCC
:1083600032EC4AF0120024D885EF41F00501DF51CC
:108370000501DA5D0501E0510501DB590AE3DCC5C1
:10838000D7F5DDC5D8F5DEC5D9F5DFC5DAF5E0C529
:10839000DBF5D7C5E1F5D8C5E2F5D9C5E3F5DAC512
:1083A000E4F5DBC5E5F50601470EBF6F32EF4AF095
:1083B0000501E469630EE56FCDEC1CF000090CE0EB
:1083C00029C631F62AC632F636EC30F0000904E050
:1083D00029C6E4F52AC6E5F517EC49F00501E16F79
:1083E000FFEC4AF00501E26FD2EC45F00501E36FC6
:1083F0001200BCDFFCEF41F00501E1510401569D84
:0E840000E8B0568DE2C557F4E3C558F41200FB
:02840E00060165
:108410004D514F1908E14E51501905E151C6F3FF76
:1084200052C6F4FF12004D514B5D0D01136F060152
:108430004E514C590D01146F156B166B06015151BD
:10844000535D146E54515255156E5BD814C00BF029
:1084500015C00CF049D88BEC49F005C0EDFF04C005
:10846000EDFF03C0EDFF02C0EFFF06014D514F5D70
:108470000D01176F06014E5150590D01186F17CDA0
:1084800014F0156ED89015321432000114500D01FD
:108490001327000115500D011423000E1523162378
:1084A00017CD14F018CD15F02CD817CD0BF018CD32
:1084B0000CF01AD8BAEC4AF009C0EDFF08C0EDFF85
:1084C00007C0EDFF06C0EFFF060151510D01132754
:1084D000060152510D011423000E1523162313CD4E
:1084E000F3FF14CDF4FF120016C00DF017C00EF00C
:1084F000EECF06F0EECF07F0EECF08F0EFCF09F0A9
:108500001200166A176A130EE96E0D0EEA6E12005B
:10851000FEEC3EF0D7EC28F0F26A10EF00F012000B
:10852000A1EC35F0000916E10601A151A21104E108
:108530003FC6A1F640C6A2F6C2EC1CF0000904E05A
:108540003FC6A1F640C6A2F6A1C6FAF0A2C6FBF04D
:10855000A9EC35F012000601A3514A0A29E0020AEB
:1085600024E00F0A1FE0010A1AE0030A15E0010ADD
:1085700010E0070A0BE0010A06E0030A01E012001E
:1085800080CF00FD17D081CF00FD14D082CF00FD39
:1085900011D083CF00FD0ED084CF00FD0BD085CF4E
:1085A00000FD08D086CF00FD05D087CF00FD02D0AA
:1085B00088CF00FD0601500E8C6FC3EC46F006011B
:1085C000500E8C6FC3EC46F0A3C68CF6C3EC46F09D
:1085D00000CD08FF57EC33F049EF33F0FEEC3EF0EE
:1085E000D7EC28F0FF0012000601C2A104D006015A
:0885F0008D890501FC8D1200CC
:0885F800060173978FA8000C27
:1086000006019E5101E0000CDC0E0401141902E188
:10861000050E151908E00401F66BF76B26EC1DF04A
:10862000000901E0000CF2EC1EF0000905E002EC8C
:1086300030F0000901E0000C8F9844D8010C8FB88D
:10864000000C06019E5122E106011C510401165D39
:1086500006011D510401175919E2DC0E141902E13B
:10866000050E151913E00601BC51BD110EE016C42C
:1086700019F517C41AF51CC617F51DC618F5BCC6A2
:1086800015F5BDC616F562EC23F0010C8F881AD8DB
:10869000010C01EC23F00601410E19D84D0E17D83C
:1086A000500E15D8490E8C6FC3EC46F08FA803D03E
:1086B0000601310E02D00601300E8C6FC3EC46F07D
:1086C00049EF33F00501005101E0E3DF12008C6F48
:0886D000C3EC46F006011200A4
:0886D800D5EF43F0235005E04B
:1086E000100E06019C6F9D6B09D011EC48F000093B
:1086F00007E10601380E9C6F010E9D6F17D814D04C
:108700000401F66BF76B26EC1DF000090DE19BEC04
:1087100046F0000909E0A3EC46F0000905E07CEC16
:108720003FF0000901E1010C40D8000C06019C510A
:108730009A5D9D519B5904E29CC69AF69DC69BF694
:10874000120062EC4BF060EC4BF0209675EC48F0B8
:108750006582D382D38E03000000D3926592F29695
:10876000C70EF01650EC4BF055EC4BF0040E060122
:108770009C6F9D6BDBDF120006019A519B1103E099
:108780009A07000E9B5B9A519B110EE1A7DF00092F
:108790000BE00601C2A103D070EC48F004D0C70E74
:1087A000F01675EC45F0CDDF1200040E06019C6F4B
:0687B0009D6B96EF43F003
:0A87B60061EC48F06CEC43F07BEC42
:1087C00048F0CCEC3EF07CEC28F071EC3FF091EC02
:1087D00036F0B0EC3CF050EC4BF055EC4BF0D08E5A
:1087E000F28CF28EF08AB7EC13F036EC1FF0ABECA3
:1087F00046F0D7EF1EF020A006D0209009EC3EF006
:10880000F08A73EC3DF0060170A30BD07093050164
:10881000E651000806E2A1EC35F0000902E105018D
:10882000E607060170A12DD070910601BE2BBE5146
:10883000146E156A1450070B11E10601738BCAEC14
:108840003AF085EC3FF079EC45F0DAEC46F0EEECEE
:1088500046F0040109AB02D0BCEC43F00601C2A112
:1088600010D0C2BD0ED006016C5103E1B4EC3CF057
:1088700008D090EC30F0040E06019C6F9D6B96ECD6
:0C88800043F0B8EC36F0D2EC47F0B5D76E
:04888C0008C012F01E
:1088900008500D02F4CF07F0F3CF06F009500E0296
:1088A000F4CF09F0F3CF08F00D02F3500726F4508F
:1088B0000822E86A092212500E02F3500726F450EB
:1088C0000822E86A0922000C09C013F008C012F05F
:1088D00007C011F007500C02F4CF05F0F3CF04F0FD
:1088E00008500D02F4CF07F0F3CF06F00C02F3505E
:1088F0000526F4500622E86A072211500D02F350B3
:108900000526F4500622E86A072209500C02F350AB
:108910000626F450072209500D02086AE86A082268
:10892000F3500726F450082211500E02F350062689
:10893000F4500722096AE86A0822092212500E023E
:10894000F3500726F4500822E86A092213500E0259
:0A895000F3500826F4500922000C31
:06895A0001EC23F0060110
:10896000540E5ED80601530E5BD823500F010C6FD6
:108970000D6BB5EC33F00501D3510F010C6F0D6B8E
:10898000B5EC33F0D4C50CFFD5C50DFF41D849EF88
:1089900033F00501005114E001EC23F00601410E13
:1089A0003FD80601550E2FD806014F0E39D83FC6C5
:1089B0000CFF40C60DFF2CD84CEC33F091EC22F0AC
:1089C0001200050100510DE001EC23F00601460EF6
:1089D0001AD892C60CFF93C60DFFB5EC33F049ECE4
:1089E00033F01200050100510DE001EC23F0060107
:1089F0004D0E09D894C60CFF95C60DFFB5EC33F0AB
:108A000049EC33F012000CD80601540E10EF45F07B
:108A1000B5EC33F029C610FF2AC611FFC4EF33F0BE
:068A20008C6FC3EF46F06D
:0A8A2600D8CFE4FFE0CFE4FFE46ED8
:108A3000DACFE4FFE9CFE4FFEACFE4FFE6529DAAF4
:108A40001AD09EAA18D0ABA203D0AB98AB8813D093
:108A5000ABA402D0AE500FD006018951EA6A000FD4
:108A6000E96E020EEA22AECFEFFF89290601885D8A
:108A700002E00601892B9DA813D09EA811D0060103
:108A80008A5106018B5D02E19D980AD006018A5148
:108A9000EA6A000FE96E010EEA22EF50AD6E8A2BF2
:108AA000F0A003D0F090F0962084F0A202D0F092D3
:108AB0002082F0A403D0F094F09A2080F2A004D099
:108AC0008150816EF2902086A6A802D0A6987F944D
:108AD000E552E5CFEAFFE5CFE9FFE5CFDAFFE55064
:0A8AE000E5CFE0FFE5CFD8FF10005E
:068AEA0091688B848B8073
:108AF0001200060173A104D0916A8B948B9012002E
:108B0000F4DF0601C2A112001CEC48F0020A04E0E6
:108B1000030A03E1919001D0919A06019E5101E070
:108B2000919C0401F66BF76B26EC1DF000091FE029
:108B3000E3EC2FF0F3CF00FDF4CF01FD0D01000EAB
:108B4000F35C030EF45801E3919E000E005D020EEB
:108B5000015901E38B94800E005D010E015901E380
:108B60008B90330E005D010E015901E391980601CF
:108B70007051040B05E0A1EC35F0000901E0120092
:108B8000040108514D0A0CE0180A09E0170A05E033
:108B9000030A01E012009196120091921200919640
:048BA000919412009A
:0C8BA4000D01136B8FB0138F8DB0138D7B
:108BB0008DB2138B8DB413898DB613878DB8138541
:108BC0008DBA13838DBC13811351120001EC23F075
:108BD00006014C0E8C6FC3EC46F0B4C608FF57EC90
:108BE00033F049EF33F0DEDF0601B46FE6EF45F016
:108BF000D9DF0601B55D01E1000CB5AF02D08F8071
:108C000001D08F90B5AD02D08D8001D08D90B5ABE5
:108C100002D08D8201D08D92B5A902D08D8401D071
:108C20008D94B5A702D08D8601D08D96B5A502D0C2
:108C30008D8801D08D98B5A302D08D8A01D08D9AF0
:108C4000B5A102D08D8C01D08D9C01D8010C0501FD
:088C5000005101E0C8DF120031
:088C580053D854D800000B0EA4
:108C60000001FF6F9DAA1ED09EAA1DD0ABA203D00B
:108C7000AB98AB881AD0ABA402D0AE5017D0060187
:108C80008951000FE96E020EEA6EAECFEFFF0601CA
:108C90008929FF0B060188190CE006018929FF0BC1
:108CA000895309D000D000002AD800D000002AD86B
:108CB00026D8000024D826D8000000009DA814D093
:108CC0009EA813D006018B5106018A1902E19D98D6
:108CD0000FD08A51000FE96E010EEA6EEFCFADFFA3
:108CE0008A29FF0B8A6F06D000D0000008D800D078
:108CF00009D800D007D800000001FF2FB3D7120019
:088D0000FEDFFDDFFCDFFBD705
:088D08004F0EAB169D9A1200FC
:108D1000AC9A9D98120006018951885DFCE088514B
:108D2000EA6A000FE96E020EEA22EFCF00FD882BFF
:108D30000D010051120006018951885D01E0000C0F
:108D400065AC000C010C06018A518B5D01E0000C42
:108D5000ACA2000C010CD8DFDBDF0601886B896B4D
:108D60008A6B8B6BAC6AAC84100EAB6E656A05C403
:108D7000AFFF9F989F9AAC8AAB8E9EAA02D0AE504E
:108D8000FCD79D8A1200ACAA14D08BC640FD0D0101
:108D9000402B06018A510D01405DFBE006018B511D
:108DA000EA6A000FE96E010EEA228CC6EFFF8B2BF8
:048DB0009D88120088
:0C8DB4000601C2B110D006018D51020B67
:108DC00003E18D51010B02E00601C28F0601C2AF23
:108DD00004D006018D938D912DD812000601C2A1F9
:108DE00013D006018DA303D08D930601C28D060119
:108DF000C2AD0AD02DEC3DF0000906E1A3EC46F02F
:108E00000009FCE00601C26B120001EC23F0060130
:108E1000500E8C6FC3EC46F00601530E8C6FC3EC02
:108E200046F00601C251010B0F010A6F6DEC33F0E1
:108E300049EF33F00601C251010B10E1C251800B22
:108E40000DE00601746B756B766B0601C26BC28117
:0E8E500006019F6B05EC3BF05EEC3DF012005E
:028E5E008FA6DD
:108E6000000C8F9646D8010C8FB6000C06011C51E1
:108E70000401205D06011D510401215910E220C4A6
:108E800019F521C41AF51CC617F51DC618F50501FC
:108E9000430E156F230E166F62EC23F0000C8F86C5
:108EA00028D8010C8FA6000C06011C510401225D7C
:108EB00006011D510401235901E3000C06017385CD
:108EC000CEDF010C01EC23F00601410E17D8540E41
:108ED00015D8540E13D84E0E8C6FC3EC46F08F503D
:108EE000080B01E0010E0F010A6F6DEC33F049EF42
:108EF00033F00501005101E0E5DF12008C6FC3EC97
:068F000046F0060112001C
:0A8F0600200EF66E080EF76E000E46
:108F1000F86E06010900F550466F0900F550476FDD
:108F200003E1466701D03DD00900F550416F0900CB
:108F3000F550426F0900F550436F09000900F550E4
:108F4000E96E0900F550EA6E090009000900F550C4
:108F5000446F0900F550456F09000900F6CF48F647
:108F6000F7CF49F6F8CF4AF641C6F6FF42C6F7FFFB
:108F700043C6F8FF0601445302E1455307E00900E8
:108F8000F550EE6E4407F8E24507F9D748C6F6FFFC
:108F900049C6F7FF4AC6F8FF06014607000E475BC1
:048FA000BFD7120025
:0C8FA400060189510601885D39E08BEC64
:108FB00046F00D01436FE85004E1000160510008E4
:108FC000F1E243CDC0F6BBEC4BF0E66E0001605120
:108FD000EA6A610FE96E000EEA22E552E750EF6E91
:108FE0006029EA6A610FE96E000EEA22EF6A950EC7
:108FF000605D01E2602B3B0E0D01435DD3E1050195
:10900000610E776F000E786FC6EC15F00001606B93
:109010000601380E9C6F010E9D6F96EC43F0C2D78F
:109020001200060189510601885D01E0000C000173
:08903000605101E0000C010C8D
:089038008FA4010C90BE030C93
:10904000020C010E0601A75D01E2000CA751030806
:1090500001E2000C010C01EC23F00601410E8C6FC3
:10906000C3EC46F006014E0E8C6FC3EC46F0300E9A
:109070000601A81106018C6FC3EC46F049EF33F0EE
:10908000DBDF0601A86F2BEF48F0D6DF0601A95DF4
:1090900001E1000CA951030A09E0010A05E0030AF5
:1090A00008E18F94909E06D0909E01D0908E8F8480
:1090B00001D0000C01D8010C0501005101E0E0DFF6
:0290C00012009C
:0E90C2000F01F40E196F550E7E6EAA0E7E6E13
:1090D0005F8B188BFD0E186F5F9B17691669120066
:1090E000F80EF016380EF01212008150816E00005A
:1090F000F290F28612000F01010E256F246B700EA4
:10910000236F050E8B6E8C6A8D6A8E6A8F6A200EB5
:10911000906E91683D0E926E3F0E936E900E946E1F
:10912000956A966A700E976E200E986E0B0E996E69
:0E9130009A6AF296F16AF18EF188F06A1200E6
:02913E0077C6F2
:1091400014F078C615F0166A1634000E161807E6E5
:10915000D880600E1454EA0E1554000E165405E221
:10916000600EF36EEA0EF46E12000601010E775DDA
:10917000000E785904E2010EF36EF46A120077C60D
:10918000F3FF78C6F4FF120001EC23F00601460E4F
:109190008C6FC3EC46F079C60CFF7AC60DFFB5ECB8
:1091A00033F049EF33F00501005105E07BC679F655
:0891B0007CC67AF6E9DF12002B
:0891B80028D896C610FF97C6E7
:1091C00011FFC4EC33F049EF33F01FD80601420E13
:1091D0008C6FC3EC46F098C610FF99C611FFC4EC23
:1091E00033F049EF33F0050100A905D029C696F602
:1091F0002AC697F6E1DF1200050100A905D02BC6AB
:1092000098F62CC699F6E1DF120001EC23F0060176
:10921000560E08D8530E06D8570E04D8520E8C6F2F
:0E922000C3EF46F08C6FC3EC46F0060112005F
:02922E008D5061
:10923000800B01E0010C000C01EC23F00601530E41
:109240002BD8490E29D8440E27D8450E8C6FC3EC75
:1092500046F00601B00503E10601410E02D0060109
:10926000540E8C6FC3EC46F049EF33F0E0DF06019B
:10927000B06F1CEF49F0DBDF0601B15D01E1000CCE
:10928000B151E8B08D8EE8A08D9E01D8010C05018A
:10929000005101E0EBDF12008C6FC3EC46F00601D9
:0292A0001200BA
:0E92A20001EC23F00601420E8C6FC3EC46F087
:1092B0000601590E8C6FC3EC46F00601500E8C6F00
:1092C000C3EC46F00601B85103E10601420E02D09C
:1092D00006014E0E8C6FC3EC46F049EF33F08F5011
:1092E000020B01E0010E0601B86F51EF49F08F50FB
:1092F000020B01E0010E0601B95D01E1000CB9515C
:10930000E8B08F82E8A08F9201D8010C05010051CE
:0693100001E0E5DF1200A0
:0A93160006500B02F3CF02F0F4CF73
:1093200003F00C02F3500326000EF420046E0650E6
:109330000D02F3500426000EF420056E06500E02B6
:10934000F350052607500B02F3500326F450042275
:10935000000E052207500C02F3500426F45005229B
:1093600007500D02F350052608500B02F350042657
:10937000F450052208500C02F350052609500B0248
:06938000F3500526120067
:0A93860001EC23F00601410E2CD883
:10939000480E2AD8340E28D84B0E8C6FC3EC46F0FA
:1093A0008BA203D00601310E02D00601300E8C6F65
:1093B000C3EC46F049EF33F00601C36BE0EF49F030
:1093C0008B50020B01E0010E0601C35D01E1000CB0
:1093D000C351E8B08B82E8A08B9201D8010C050143
:1093E000005101E0D0DF12008C6FC3EC46F00601A3
:0293F000120069
:0E93F2003FC663F640C664F647EC3AF00D0144
:10940000206F040103510D01205D08E1E6EC3DF001
:10941000F3CFAAF6F4CFABF613D80FD02051050145
:10942000196F1A6B3FC617F540C618F50501720E85
:10943000156F1F0E166F62EC23F00F0E236E1200D5
:109440000601AA51AB1108E090EC10F0AAC687F310
:0A945000ABC688F362EC14F01200C2
:06945A000501005101E0D4
:109460001FD81200050100511AE001EC23F0BFC61D
:109470008CF6C3EC46F00601420E1ED8450E1CD8F1
:10948000530E1AD8540E8C6FC3EC46F0E4C510FF8F
:10949000E5C511FFC4EC33F04CEC33F001D81200F9
:1094A000E1C5B0F61CEC49F0E2C5B6F601EC4BF0B4
:1094B000E3C5B4F6E6EF45F08C6FC3EC46F0060169
:0294C000120098
:0E94C2001ED881C679F682C67AF6C4EF48F04D
:1094D0000501005101E0F5DF1200050100510FE028
:1094E0000FD87EC60BFFB0EC33F07DC60BFFB0EC9F
:1094F00033F07FC60BFFB0EC33F049EC33F01200D1
:1095000001EC23F00601410E8C6FC3EC46F006011E
:10951000550E8C6FC3EC46F00601580E8C6FC3EFEE
:0295200046F013
:0E952200300E0601E76EB219E8AE02D0E73453
:1095300002D0E750B25D01E2000C330EE76EB219C3
:10954000E8AE02D0B23503D0E750D880B25501E280
:10955000000C010C0601420E8C6FC3EC46F00601B4
:10956000520E8C6FC3EC46F0B3C68CF6C3EC46F0DB
:0495700049EF33F09C
:0C957400056A046A036A026A200EE76EB2
:10958000D8900636073608360936023603360436D2
:1095900005360B50025C0C5003580D5004580E5009
:1095A000055809E30B50025E0C50035A0D50045A43
:0C95B0000E50055A062AE72EE4D71200E0
:0495BC000601A651AD
:1095C000A4250D01406F000E0601A5210D01416F7C
:1095D000426B40510601A45D0D0141510601A559A0
:1095E0000BE2A4C6E9FFA5C6EAFFA42B000EA52343
:0E95F000EF500D014227EDD70D014251120040
:0295FE008C508F
:10960000120001EC23F00601430E8C6FC3EC46F010
:10961000B6C608FF57EC33F049EF33F08CCFB6F6FF
:1096200001EF4BF00601B7518C5C01E1000CB7C6AD
:109630008CFF01D8010C0501005101E0EFDF1200A1
:10964000FE0EE3CFE9FFFF0EE3CFEAFFE9CFF3FF22
:10965000EACFF4FFFB0EE35003E1FC0EE35009E018
:10966000FB0EE30602E2FC0EE306FD0EE350EE6E97
:04967000F1D712001C
:0C967400056A046A100EE76ED8900836F4
:109680000936043605360D50045C0E50055805E3C6
:109690000D50045E0E50055A082AE72EF0D712002E
:1096A000D76AD66AA10ED56E1200060ECD6E9E90B8
:1096B0009F809D80E00ECF6EC60ECE6ECD801200D4
:0C96C000D56A12009D90CD909E90120083
:0496CC000601BB5187
:1096D000030A0AE0010A05E0030A08E1BAA106D07C
:0E96E000010CBAA303D0010CBAB5010C000CAA
:0296EE001EEE6E
:1096F00000F02EEE00F0F86A019C87EC4BF083EC52
:0E97000047F0DBEC43F0FBEC43F0FBD712002C
:02970E00160E35
:10971000F36E00EE00F00F0E01D81200EA6002D0E6
:0E972000EE6AFCD7F350E9601200EE6AFCD747
:02972E00056ACA
:10973000080EE76ED890093605360E50055C02E338
:0A974000056E092AE72EF7D7120084
:06974A000010303AD84681
:10975000484F60648080A09CB0AAD0C6E8DBC8EC0B
:109760006C07A60EF714EE1B8D275F37C646E9522D
:069770006C61B27020CB19
:0A977600610E0601C05D05E3C0515D
:0C9780007A0802E3200EC05FC051120006
:01978C007E5E
:03978D00B80BC056
:109790001270172823C8326842384AD85990657029
:0397A00094FFFF34
:020000040030CA
:0100000015EA
:0100010002FC
:0100020056A7
:010003001CE0
:01000400F902
:010005008179
:010006008178
:01000800FFF8
:01000900C036
:01000A00FFF6
:01000B008074
:01000C00FFF4
:01000D0040B2
:00000001FF
